:100000000C94A9020C94C6020C94C6020C94C6026D
:100010000C94C6020C94C6020C94C6020C94C60240
:100020000C94C6020C94C6020C94C6020C94C60230
:100030000C94C6020C94C6020C94C6020C94C60220
:100040000C94122E0C94C6020C94C6020C94C60298
:100050000C94C6020C94C6020C94C6020C94C60200
:100060000C94C6020C94C602312E30362E3030006D
:100070004845414400474554202F0054532D4E54C9
:1000800050434B30315F58585858006E74702E6A88
:1000900073742E6D666565642E61642E6A70006EE1
:1000A00074702E6E6963742E6A70008B009F00213D
:1000B0000441043031323334353637383941424324
:1000C00044454600485454502F312E3120323030B0
:1000D00020485454500D0A436F6E6E656374696F07
:1000E0006E3A20636C6F73650D0A436F6E74656EB4
:1000F000742D547970653A20746578742F68746D26
:100100006C0D0A43616368652D436F6E74726F6C8A
:100110003A206E6F2D63616368650D0A436F6E74DC
:10012000656E742D4C616E67756167653A20656E0A
:100130000D0A0D0A00485454502F312E3120323010
:1001400030204F4B0D0A436F6E6E656374696F6E9E
:100150003A20636C6F73650D0A436F6E74656E743D
:100160002D547970653A20746578742F68746D6CBD
:100170000D0A43616368652D436F6E74726F6C3A4C
:10018000206E6F2D63616368650D0A436F6E746541
:100190006E742D4C616E67756167653A20656E0DF2
:1001A0000A0D0A3C21444F43545950452048544DB0
:1001B0004C205055424C494320222D2F2F5733437A
:1001C0002F2F4454442048544D4C20342E3031209D
:1001D0005472616E736974696F6E616C2F2F454E36
:1001E000222022687474703A2F2F7777772E773316
:1001F0002E6F72672F54522F68746D6C342F6C6F92
:100200006F73652E647464223E3C48544D4C3E3CF2
:10021000484541443E3C5449544C453E54532D4E70
:1002200054502D434C4F434B2053455455503C2F75
:100230005449544C453E3C2F484541443E3C424F76
:100240004459204247434F4C4F523D222346464695
:100250004646464646223E3C43454E5445523E3C69
:10026000423E00223E3C2F464F524D3E3C42523EC3
:100270003C464F4E5420434F4C4F523D224752452F
:10028000454E223E56414C55452053415645443C2F
:100290002F464F4E543E3C42523E00223E3C42527C
:1002A0003E3C42523E3C494E5055542054595045D4
:1002B0003D225355424D4954222056414C55453D0F
:1002C000224150504C59223E3C2F464F524D3E0049
:1002D0004E31004E3200D002D302534552564552A1
:1002E00031005345525645523200DA02E2024000D4
:1002F00060006E732E6367690066617669636F00E4
:10030000F202F90254494D452053455256455220B8
:1003100053455454494E470020485454502F003CF4
:1003200042523E3C2F43454E5445523E3C2F424F95
:1003300044593E3C2F48544D4C3E0022204D4554DC
:10034000484F443D22474554003C2F423E3C4252D8
:100350003E3C464F524D20414354494F4E3D2200B2
:10036000222056414C55453D220022204D41584CFB
:10037000454E4754483D2200222053495A453D22CC
:10038000003C42523E3C494E505554205459504531
:100390003D225445585422204E414D453D220022D5
:1003A0003E3C42523E0054494D4552204F46460085
:1003B00053494E474C45204D4F444500434F4E5402
:1003C000494E5545204D4F444500A603B003BC039C
:1003D0000209000509000509534D545754465300BE
:1003E0002D2D2054494D4552204D4F4445202D2D53
:1003F000004F464654494D45004F4E54494D450027
:1004000020203A20203A2020004F464620574441E1
:10041000593A004F4E2020574441593A0053554E07
:10042000004D4F4E00545545005745440054485523
:100430000046524900534154004149555454532DEC
:100440004E54502D434C4F434B303100454E4332B8
:10045000384A3630205245563A00494E49544941AF
:100460004C495A494E472E2E2E00494E4954494177
:100470004C495A4544004B4559494E505554204922
:100480004C4C4547414C0043414C2052454D3A00AD
:100490003D044C045A046A0476048704566572735A
:1004A000696F6E00504C4541534520434845434BCE
:1004B000204B455900504C4541534520524553452A
:1004C00054004D41433A0044484350434E543A008F
:1004D00054494D45523A009C04A404B504C204C7D3
:1004E00004D004455850495245442000205245420A
:1004F000494E44200052454E4557414C2000494E3C
:1005000046494E49545900E304EC04F504FE042D19
:100510002D2F2D2D202D2D3A2D2D3A2D2D004F46EE
:10052000460053474C00434E54001E052205260545
:10053000C0F9A4B0999282F88090FF88FBC1872A05
:100540002A3A2A2A3A2A2A002D2D3A2D2D3A2D2DE3
:10055000000011241FBECFEFD8E0DEBFCDBF12E0F8
:10056000A0E0B1E0EAE7FEE702C005900D92AA36EE
:10057000B107D9F715E0AAE6B2E001C01D92A53E89
:10058000B107E1F70E9448050C943B3F0C94000032
:100590006091BA05262F30E08091230190912401CB
:1005A00028173907C9F55091BB05252F30E08091F8
:1005B0002101909122012817390771F54091BC055E
:1005C000242F30E080911F019091200128173907D6
:1005D00019F55F9A8091B6058130F1F48091BE05DE
:1005E0006817A1F48091BF05581781F48091C00568
:1005F000481761F41092B60501C0A895F999FDCF8E
:1006000085E390E060E00E94F83E089581E090E08C
:100610009093B8058093B70508958091BE0590E04A
:1006200020912301309124018217930721F58091B5
:10063000BF0590E02091210130912201821793079C
:10064000D1F48091C00590E020911F0130912001EC
:100650008217930781F45F988091B605813059F431
:100660001092B60501C0A895F999FDCF85E390E0F9
:1006700060E00E94F83E0895A0E2B0E0E2E4F3E01A
:100680000C94FF3D0E949E0D82E00E94F13301C058
:10069000A895F999FDCF8EE090E060E570E00E94AA
:1006A000363F01C0A895F999FDCF8CE090E06AE053
:1006B00070E00E94363F01C0A895F999FDCF85E30F
:1006C00090E060E00E94203F01C0A895F999FDCF1D
:1006D00086E390E040E050E060E070E00E942E3F52
:1006E00001C0A895F999FDCF8AE390E040E050E081
:1006F00060E070E00E942E3F01C0A895F999FDCFFF
:100700008E010F5F1F4FC8016BE870E00E944D3EE5
:10071000C80160E470E040E250E00E94163F01C072
:10072000A895F999FDCF8E010F5F1F4FC8016FE9A2
:1007300070E00E944D3EC80160E670E040E250E08B
:100740000E94163F01C0A895F999FDCF80EC90E07A
:1007500068E572E00E94363F01C0A895F999FDCF87
:1007600082EC90E06CED75E00E94363F01C0A895E8
:10077000F999FDCF8EE390E065EA73EC0E94363F75
:10078000A096E4E00C941B3EA4E0B0E0EAECF3E0B9
:100790000C94FF3D8E010F5F1F4FC80160E00E9467
:1007A00071238130B1F489819A81AB81BC8100973A
:1007B000A105B10571F4C80161E00E947123813087
:1007C00041F489819A81AB81BC810097A105B10573
:1007D00039F081E090E090930A018093090104C010
:1007E00010920A01109209012496E4E00C941B3E39
:1007F0000E945C0F89B180958770873069F40E94F0
:100800003C030E949E0D83E00E94F13382E00E942F
:10081000E433A895FECFA895F999FDCF8EE390E03B
:100820000E94E23E855A934C21F00E943C0301C095
:10083000A895F999FDCF8EE090E00E94E23E90935A
:1008400014038093130301978E5F9F4F30F080E570
:1008500090E0909314038093130380E10E943A0F79
:100860006093DA027093DB028093DC029093DD02E6
:1008700082E10E943A0F6093DE027093DF02809360
:10088000E0029093E10284E10E943A0F6093E20259
:100890007093E3028093E4029093E50286E10E9464
:1008A0003A0F6093A3057093A4058093A5059093D8
:1008B000A60501C0A895F999FDCF8CE090E00E94B3
:1008C000E23E9C013F773093BC042093BB04019728
:1008D0008E5F9F4F30F08CE390E09093BC04809348
:1008E000BB048091DA029091DB02A091DC02B0910E
:1008F000DD020097A105B105B9F48091DE02909167
:10090000DF02A091E002B091E1020097A105B105DC
:1009100059F48091AB059091AC05019711F084E1F9
:1009200001C085E18093BE0483E995E06BE770E048
:100930000E944D3E809104016EE975E00E94142CE6
:100940008091050160EA75E00E94142C01C0A89511
:10095000F999FDCF85E390E00E94D43E8093B605DF
:1009600001C0A895F999FDCF86E390E00E94DC3E96
:100970006093B9057093BA058093BB059093BC054D
:1009800001C0A895F999FDCF8AE390E00E94DC3E72
:100990006093BD057093BE058093BF059093C0051D
:1009A00080E490E061E274E04BE850E00E94CC0EFD
:1009B00080E690E061E474E04FE950E00E94CC0EE4
:1009C0000E94C40301C0A895F999FDCF80EC90E086
:1009D0000E94E23E909382048093810401978E5F8F
:1009E0009F4F40F088E592E09093820480938104C9
:1009F00001C0A895F999FDCF82EC90E00E94E23EFB
:100A000090938604809385048F5F9F4F31F48CED23
:100A100095E090938604809385041092AF05089525
:100A2000EF92FF920F931F93E0908304F090840461
:100A30000027F7FC0095102F83E491E06FE171E04F
:100A40000E94C32DE61AF70A080B190BB701C8015B
:100A50001F910F91FF90EF9008950F931F938C01BA
:100A60000E94B52C005110406F717070600F711FA3
:100A70007093840460938304A3E4B1E0EFE1F1E0B8
:100A800082E101900D928150E1F71F910F9108953D
:100A9000A4E0B0E0EEE4F5E00C94F13DF8948BECCA
:100AA0008093640080E880BF14E015B918B880E630
:100AB0008BB98FE284B98FE387B980EF8AB988E078
:100AC00090E00E94DC3E60938704709388048093DA
:100AD000890490938A0480E18CBD16BC14BC15BDBA
:100AE00081E080936E0084B7992787FD909580FD03
:100AF0000CC081FD04C082FD02C083FF06C081E0FE
:100B000090E09093AC058093AB0514BE2CE088E197
:100B100090E00FB6F894A895809360000FBE2093E4
:100B20006000789410E51CBD0E941D3380E18CBDEF
:100B30000E94F70D0E94F8031CBD299A89E190E0FC
:100B40000E94370E0E94AF09882331F484E162EAE3
:100B50007AE00E94DE08FFCF0E94170C8EE190E041
:100B60000E94460E80E00E94F13380E00E94E43350
:100B700088E061E048E650E00E94CF0D8EEE92E002
:100B80000E94460E0E949E0D8091BE048823D1F0E3
:100B900081E090E09093C0048093BF04ABE0B1E0AB
:100BA000EFE1F1E082E101900D928150E1F7809157
:100BB000BE04843119F40E94C61908C086E10E945F
:100BC000A41A04C01092C0041092BF041092AC0585
:100BD0001092AB050E943E0E5C014E010894811CF0
:100BE000911C61E0662E712C01E05CE3452E512CD6
:100BF00042E0342E30EC232EA8950E94C61382309A
:100C000019F40E94421209C0833019F40E94A518F9
:100C100004C0843009F50E941216182F0E94380A69
:100C20001123D1F0163091F48091B0058823A1F002
:100C3000A3E4B1E0EFE1F1E082E101900D92815097
:100C4000E1F7109290051092B00506C01B3121F417
:100C500080E490E00E942D05F8948091C705909162
:100C6000C8059093AE058093AD051092C80510920B
:100C7000C7057894019709F026C1F8948091C305BF
:100C80009091C405A091C505B091C60589839A834A
:100C9000AB83BC837894C4010E94DC0F9C01009755
:100CA00029F420920701009306019AC0A1E3B1E064
:100CB000FC0182E101900D928150E1F780910701E2
:100CC0008034D9F58091B105882309F073C08091F3
:100CD000350190913601892B09F06CC08091330168
:100CE00090913401892B09F065C080913101909178
:100CF0003201892B09F05EC089819A81AB81BC8168
:100D00000197A109B10989839A83AB83BC83809140
:100D1000C3059091C405A091C505B091C605019782
:100D2000A109B1098093C3059093C405A093C5059B
:100D3000B093C6053092B105A0C18038D9F5809135
:100D4000B1058823B9F58091350190913601479717
:100D500089F58091330190913401CB9759F58091B9
:100D6000310190913201CB9729F589819A81AB812C
:100D7000BC810196A11DB11D89839A83AB83BC837D
:100D80008091C3059091C405A091C505B091C60599
:100D90000196A11DB11D8093C3059093C405A09336
:100DA000C505B093C6050093B10567C10093060160
:100DB0001092A805C9016FE171E00E94E02D8091B9
:100DC000B105813029F4109207011092B10508C0D5
:100DD000823031F45092200140921F010093B105FE
:100DE0000E9435100E94CB210E94A71B809109010F
:100DF00090910A010197E1F48091B0058823C1F434
:100E00000E9410056B017C011616170618061906BC
:100E100094F08091DA029091DB02A091DC02B09113
:100E2000DD020097A105B10531F00093B00503C0C4
:100E3000CC24DD2476018091B605882311F1813020
:100E400059F48091B7059091B805019711F40E946B
:100E50000D030E94C80215C0C30100902B0102C0FF
:100E6000880F991F0A94E2F7182F8091B905812302
:100E700011F00E94C8028091BD05182311F00E9454
:100E80000D038FE191E00E9429338091A70588230B
:100E900019F40E94BC3417C08430A9F48091090170
:100EA00090910A01892B21F08091B005882321F0CF
:100EB00080E00E94DD3305C080E0B701A6010E94FA
:100EC00032340E947C348091A805882311F181304E
:100ED000E1F480918304909184048034910514F4AA
:100EE00080E490E0880F991F24E08130920714F08D
:100EF00080E094E00E942D05A3E4B1E0EFE1F1E091
:100F000082E101900D928150E1F71092B0051092AC
:100F10000601809190058823B9F00E941C22882345
:100F2000C9F080518B3058F4A3E4B1E0EFE1F1E077
:100F300082E101900D928150E1F70E948E23109280
:100F400090051092B00506C010928F051092920580
:100F5000109291050E942D24882341F01092900553
:100F60001092B00580E490E00E942D058091AD05BF
:100F70009091AE050197F1F48091EF02882359F02A
:100F800080910003815080930003882321F480E046
:100F900090E00E94D71580910103882359F0809139
:100FA0001203815080931203882321F481E090E0A2
:100FB0000E94D7158091A9059091AA05019711F477
:100FC0000E9455351092AA051092A9051092AE05FF
:100FD0001092AD051092A8050E943E0E8A199B0939
:100FE000059740F10E943E0E5C010E945B0E0E943C
:100FF0006A0E8823F9F01091A705813121F41F5F53
:10100000153098F413C0833119F40E9485310DC056
:10101000843119F40E94F70D09C0853111F45F9AEB
:1010200009C0863139F45F9805C010E01093A70518
:101030000E94553580910601882331F47092B305E2
:101040006092B2055D9805C01092B3051092B2058A
:101050005D9A8091DA029091DB02A091DC02B0915E
:10106000DD020097A105B10531F00E94F009813041
:1010700011F45E98C1CD5E9ABFCDC4010E94DC0F11
:101080009C01A1E3B1E0FC0182E101900D9281504D
:10109000E1F72115310509F08DCE88CE8EBD0DB456
:1010A00007FEFDCF08952A988EBD0DB407FEFDCF33
:1010B0001EBC0DB407FEFDCF8EB52A9A08952A985E
:1010C0008EBD0DB407FEFDCF1EBC0DB407FEFDCFD7
:1010D0008EB51EBC0DB407FEFDCF8EB52A9A0895BD
:1010E0002A98805C8EBD0DB407FEFDCF6EBD0DB499
:1010F00007FEFDCF2A9A08950F931F93182F0E9481
:101100005F08082F812F8F5F0E945F08982F802F24
:101110001F910F9108950F931F93182F072F0E946F
:101120007008812F8F5F602F0E9470081F910F91B0
:1011300008952A9880588EBD0DB407FEFDCF6EBD70
:101140000DB407FEFDCF2A9A08952A9880568EBDC9
:101150000DB407FEFDCF6EBD0DB407FEFDCF2A9A7C
:1011600008951F93182F8FE163E00E94A5088FE177
:10117000612F0E9499081F9108951F93182F82E0F4
:101180000E94B10884E1612F0E94700882E161E051
:101190000E94700883E00E94B1088AE00E945F0804
:1011A00080FDFBCF82E00E94B10882E160E00E94F6
:1011B000700888E10E947C081F910895FF920F93A8
:1011C0001F93F82E8B0182E00E94B10884E16F2DFD
:1011D0000E94700886E1B8010E948B0883E00E949B
:1011E000B1088AE00E945F0880FDFBCF1F910F913C
:1011F000FF9008952A988AE38EBD0DB407FEFDCFB7
:101200001EBC0DB407FEFDCF8EB52A9A08952A980C
:101210008AE38EBD0DB407FEFDCF1EBC0DB407FEE4
:10122000FDCF9EB51EBC0DB407FEFDCF8EB52A9A2C
:1012300008952A988AE38EBD0DB407FEFDCF1EBC2B
:101240000DB407FEFDCF9EB51EBC0DB407FEFDCF4D
:101250008EB51EBC0DB407FEFDCF7EB51EBC0DB411
:1012600007FEFDCF6EB52A9A0895FC012A988AE3FD
:101270008EBD0DB407FEFDCF20E030E008C01EBCDF
:101280000DB407FEFDCF8EB581932F5F3F4F26171C
:101290003707A8F32A9A0895982F2A988AE78EBDCF
:1012A0000DB407FEFDCF9EBD0DB407FEFDCF2A9AFB
:1012B0000895282F2A988AE78EBD0DB407FEFDCF2A
:1012C0009EBD0DB407FEFDCF2EBD0DB407FEFDCFB4
:1012D0002A9A0895282F2A988AE78EBD0DB407FE12
:1012E000FDCF9EBD0DB407FEFDCF2EBD0DB407FE94
:1012F000FDCF7EBD0DB407FEFDCF6EBD0DB407FE64
:10130000FDCF2A9A0895FC012A988AE78EBD0DB474
:1013100007FEFDCF20E030E008C080818EBD0DB417
:1013200007FEFDCF2F5F3F4F319626173707A8F3F3
:101330002A9ACB010895282F2A988AE78EBD0DB4EA
:1013400007FEFDCF80E090E005C02EBD0DB407FE86
:10135000FDCF019686179707C0F32A9A08950F9339
:101360001F938FE160E00E94700880E160E070E010
:101370000E948B0882E16FEF7FE10E948B088AE078
:101380006FEF7FE10E948B0883E00E94B10887E045
:1013900067E00E94700887E00E94530880FDFBCF41
:1013A00087E062E00E94A5088FE160E30E9499084F
:1013B0008FE10E94530885FDFBCF80E00E94B108B9
:1013C00086E10E945308082F87E10E945308182FD6
:1013D00080E00750184F09F481E01F910F910895A4
:1013E00081E00E94BD0896958795969587958170B6
:1013F0000895EF92FF920F931F938C0180E00E945B
:10140000B10880E00E947C08F82EE92E60917802F5
:10141000709179026A5F7F4F600F711F89E1683DAB
:10142000780710F0685D794180E00E948B088F2D6D
:101430009E2D1F910F91FF90EF900895EF92FF92D4
:101440000F931F938C0180E00E94B10882E00E94FC
:101450007C08F82EE92E0752164E82E0B8010E9451
:101460008B088F2D9E2D1F910F91FF90EF90089567
:101470000F931F9300917A0210917B02015010404C
:1014800080E00E94B1088EE160E40E949908B801F2
:1014900089E1083D180710F067ED79E18CE00E94C2
:1014A0008B081F910F910895A7E0B0E0EAE5FAE0FC
:1014B0000C94F93D8C01E0907D02F0907E02E80EE4
:1014C000F91E82E0B8010E948B0880E00E944C095E
:1014D00084E0B8010E948B0886E0B7010E948B0867
:1014E0008FE160E80E9499088FE160E80E94A508FA
:1014F0008CE16AE00E94A5088FE168E00E949908EB
:1015000080917C028550823008F068C000E010E0D5
:101510008CE10E9453088A7031F40F5F1F4F83E003
:10152000083E1807A9F78CE10E94530881FD05C009
:1015300083E0083E180708F451C08FE168E00E947C
:10154000A50880E00E947C085C0186E00E947C087F
:101550006C010894C11CD11C80E0B6010E948B086C
:101560008E010F5F1F4FC80167E070E00E943509D0
:10157000EE24F02E012F8CE10E94530881FF2AC037
:101580008C8185FF27C08FE160E80E9499088FE178
:1015900060E80E94A5088CE16AE00E94A5088FE13E
:1015A00068E00E9499088CE10E9453088A70D9F380
:1015B0008FE168E00E94A50880E0B6010E948B08D8
:1015C0008F2D902F67E070E00E943509E39480E151
:1015D000E81689F680E0B5010E948B082796EAE0BC
:1015E0000C94153EA0E0B0E0E8EFFAE00C94FA3D70
:1015F000B82E282F392F6901EE24FF24870111C04E
:101600000E94FA08D82F0E94FA08C82FCE01A0E045
:10161000B0E0E80EF91E0A1F1B1F8EEF9FEFC80EE9
:10162000D91E92E0C916D10458F7C701D8019C0110
:10163000AD01B0FE0BC00E94FA08D82FC0E09E0199
:1016400040E050E02E0D3F1D401F511F203080E034
:10165000380781E0480780E05807A0F0CA0140E061
:1016600050E0A0E0B0E0280F391F4A1F5B1F203078
:1016700090E0390791E0490790E0590718F0C90157
:1016800001969C01C901CDB7DEB7E9E00C94163E86
:101690000F931F938B010E94F909C8010E94F20A5F
:1016A0009C0120953095C9011F910F910895EF92EB
:1016B000FF920F931F938C017B0180E00E94B10881
:1016C0000752164E80E0B8010E948B08C7010E94A5
:1016D000F20A9C0120953095C9011F910F91FF904E
:1016E000EF900895A0E0B0E0E8E7FBE00C94FB3D4C
:1016F0006C017B018A014115510509F444C0413058
:10170000510551F40E94F909C7010E941E0A0E9466
:10171000FA080E944C0937C080E00E94B108C091CD
:101720007802D09179022696CC0DDD1D89E1C83D65
:10173000D80710F0C85DD94180E1BE010E948B0836
:10174000B801615070406C0F7D1F99E1683D7907C9
:1017500010F0685D794182E10E948B0889ED99E182
:10176000E80EF91E84E1B7010E948B088FE160E169
:101770000E94A5088FE160E20E9499088FE10E9413
:10178000530885FDFBCFCDB7DEB7E8E00C94173EDC
:10179000FC012A988AE38EBD0DB407FEFDCF20E040
:1017A00030E00AC01EBC0DB407FEFDCF8EB581939C
:1017B0002F5F3F4F841719F02617370798F31082D1
:1017C0002A9AC90108950F931F93CF93DF938C0139
:1017D000C0E0D0E003C00E94FA082196C017D107EC
:1017E000D0F3DF91CF911F910F910895CF93DF93A5
:1017F000EC010E94543EAC012A988AE78EBD0DB4DC
:1018000007FEFDCF20E030E00AC0FE01E20FF31F2B
:10181000E491EEBD0DB407FEFDCF2F5F3F4F2417BF
:10182000350798F32A9ACA01DF91CF9108951F9343
:101830008EE160E20E94A50889E190E00E94370EE7
:10184000299889E190E00E94370E299A89E190E079
:101850000E94370E1FEF2A981EBD0DB407FEFDCF64
:101860002A9A89E190E00E94370E8DE10E94530888
:1018700083FDF1CF80FFEFCF8FE160EC0E94700815
:101880008EE160E80E94700888E060E070E00E94ED
:101890008B088CE067ED79E10E948B088AE067EDA8
:1018A00079E10E948B0884E068ED79E10E948B0861
:1018B00081E00E94B10888E161EA0E94700882E03C
:1018C0000E94B10880E06DE00E94700881E060E055
:1018D0000E94700882E062E30E9470088AE06EEE67
:1018E00075E00E948B0886E062E17CE00E948B0834
:1018F00084E062E10E94700883E060E40E94700866
:1019000089E06FE30E94700883E00E94B10885E1DE
:1019100060E00E94700884E0609100010E947008FD
:1019200085E0609101010E94700882E060910201EF
:101930000E94700883E0609103010E94700880E0BB
:10194000609104010E94700881E0609105010E948D
:10195000700882E10E9453088F7180937C0280E0BE
:1019600060E070E00E94DE0880E160E071E00E94CB
:10197000DE0884E162E774E00E94DE0880E00E94F5
:10198000B1088FE164E00E9470081F910895CF9321
:10199000DF93EC0181E00E94B10889E10E945308C5
:1019A000882321F40E94B10880E044C080E00E94B6
:1019B000B10860917A0270917B0280E00E948B08EE
:1019C00080917A0290917B029093790280937802C1
:1019D00082E792E066E070E00E9435098091730230
:1019E0008F7180937302809175028F71809375025D
:1019F000209172023091730230937B0220937A021D
:101A000080917402909175028F5E954080F489E117
:101A1000283D380760F420FD0AC08091770287FDD9
:101A200006C08091760284FD02C087FD06C00E9438
:101A3000170C82E0DF91CF910895F8948091C3054F
:101A40009091C405A091C505B091C605809373041B
:101A500090937404A0937504B09376048091C105AB
:101A60009091C20590937C0480937B047894CE017E
:101A70006EE070E00E94350981E0DCCF98B18F7094
:101A8000907F892B88B90895449898B18F70907F82
:101A9000892B88B90000459A86E090E00E94370EB5
:101AA000459808951F93182F88B1912F92959F7094
:101AB000807F982B98B9459A86E090E00E94370E77
:101AC000459888B11F70807F812B88B9459A86E040
:101AD00090E00E94370E45981F910895449A0E9405
:101AE000520D089544980E94520D08950E946E0D63
:101AF00081E090E00E94370E0895CF93DF93EC01D0
:101B000003C021960E94760D88818823D1F7DF914A
:101B1000CF91089580E10E94720D81E090E00E94D3
:101B2000370E0895882311F48CE001C08EE00E94E6
:101B3000720D81E090E00E94370E089581E00E94CE
:101B4000720D86E290E00E94370E0895662349F0F8
:101B5000613011F4805C05C0623011F48C5E01C00C
:101B60008C5A80680E94720D81E090E00E94370ECE
:101B700008950F931F93042F0E94A60D10E004C038
:101B800080E20E94760D1F5F1017D4F31F910F9112
:101B90000895682F80E040E10E94B90D0895CF9329
:101BA000DF93EA010E94A60D03C00E94760D2196E4
:101BB000FE0184918823C9F7DF91CF9108950F9397
:101BC0001F938A010E94A60DC8010E947D0D1F91DE
:101BD0000F9108951F93142F0E94A60D812F0E942C
:101BE0006E0D81E090E00E94370E1F9108958CE009
:101BF00090E00E94460E83E00E94440D85E690E04E
:101C00000E94370E83E00E94440D81E090E00E9424
:101C1000370E83E00E94440D81E090E00E94370E71
:101C200082E00E94440D81E090E00E94370E88E23D
:101C30000E94720D81E090E00E94370E88E00E94C1
:101C4000720D81E090E00E94370E81E00E94720DDB
:101C500086E290E00E94370E86E00E94720D81E0DD
:101C600090E00E94370E8CE00E94720D089528ECDF
:101C700000002A95E9F70197D1F70895F89420918B
:101C80006A0230916B027894C9010895AC01F8940E
:101C900020916A0230916B02789401C0A895F89463
:101CA00080916A0290916B027894821B930B841747
:101CB0009507A0F308959091700289B1ECE6F2E0E7
:101CC000E90FF11D8095877080839F5F93709093DB
:101CD0007002089590916D0280916C02982380911A
:101CE0006E02982380916F02982331F1913011F4A4
:101CF00041E115C0923011F442E111C0943011F469
:101D000043E10DC0953011F444E109C0933011F462
:101D100045E105C0963011F040E001C046E1242FB6
:101D200030E08091C905992787FD909528173907DC
:101D300029F04093C90503C01092C90540E0842FE3
:101D40000895EF92FF920F931F93CF93DF93F89430
:101D5000E0906A02F0906B0278948701A895F8945D
:101D6000C0916A02D0916B027894CE01801B910BD6
:101D7000059718F00E945B0E8E010E946A0E882360
:101D800031F4CE19DF09C95BDB4040F387E1CDB701
:101D9000DEB7E6E00C94193E0F931F93CF93DF93C9
:101DA0009C01EB018A0101C0A895F999FDCFCE01F4
:101DB000B9014FE150E00E94C43E1F8E88819927EF
:101DC00087FD90950E94283E892B21F4CE01B80111
:101DD0000E944D3EDF91CF911F910F910895000019
:101DE000000000000000000008952B9A2D980000CC
:101DF00000000000000000002D9A90E087FF02C064
:101E00002B9A01C02B982D980000000000000000C4
:101E100000002D9A9F5F983011F0880FEFCF089542
:101E2000F8942D9A289A8F7380680E94F50E80E0AE
:101E300020E030E02D9800000000000000000000CD
:101E40002D9A00000000000000000000220F331F48
:101E50001C9921608F5F803169F7932F28987894BF
:101E600080917102813021F4822F0E94262D9C01E5
:101E7000C9010895CF92DF92EF92FF921F93182F1E
:101E80000E94100F6C01812F8F5F0E94100F7C0148
:101E90008FEFC8168FEFD8068FEFE8068FEFF806A2
:101EA00019F4CC24DD247601B601C7011F91FF90FF
:101EB000EF90DF90CF9008951F93CF93DF9380E052
:101EC0000E94100F8050904419F481E080937102B9
:101ED00082E00E94100F8F5F9F4F61F012E0C0E020
:101EE000D1E0812F0E94100F8883998322961F5F73
:101EF0001530B9F7DF91CF911F9108951F1D1F1E57
:101F00001F1E1F1F1E1F1E1FCF93DF93EC012C9659
:101F10004AE834D06627772736E4AEE6B1E0532F9F
:101F2000537009F01197321729F078F56A0F7B1F6B
:101F30003395F3CF4CE022D0ECEFFEE130E0C895D2
:101F40003196313011F451110A94321720F4600D9A
:101F5000711D3395F4CF402D439510D02150A8F03A
:101F6000620F711D8827992748E108D015D04CE3EE
:101F700005D012D02CE302D00FD00BC03A912A9199
:101F80002417310540F00F900F906FEF7FEF8FEF28
:101F90009FEFDF91CF91089551E2AA1B08F4A40F9F
:101FA000A79597958795779567955A95B9F7620F95
:101FB000711D811D911D0895CF93DF93FC01208138
:101FC000318142815381CC27DD2757FD3CC0CAECCB
:101FD000D5E06CE33CD00882198239D00A821B829A
:101FE00068E135D00C821D82F9012C5F3F4F67E01C
:101FF0002ED00C861D869F01A6E4EEE6F1E0BA2FF6
:10200000B37009F031972E173F0720F02E1B3F0BBE
:10201000A395F3CFAA871B862E873F87ECEFFEE1BF
:10202000AA27C8953196A13011F4B1110A94201550
:10203000310520F020193109A395F3CFA88719861F
:1020400023952E833F83CE01DF91CF910895002405
:1020500070E2220F331F441F551F001C061610F09C
:10206000061A23957A95A9F70895EFEAF2E082819E
:10207000813041F480819181019791838083892B04
:1020800009F412823D9682E0E33EF80781F7089555
:10209000CF92DF92EF92FF920F931F936B017C011F
:1020A0008AE290E090937E0280937D0280E00E941D
:1020B000B10882E06DEC7FE10E948B088FEF66E053
:1020C00070E00E949B0900E011E0C80166E070E04A
:1020D0000E94830986E098E00E94590981E090E01F
:1020E0000E94590980E098E00E94590986E00E9408
:1020F0004C0984E00E944C0981E090E00E9459095B
:10210000C80166E070E00E9483096091DA02709174
:10211000DB028091DC029091DD020E946A0980E07E
:1021200066E070E00E949B09C701B6010E946A093F
:102130008CEC9FE10E94540A1F910F91FF90EF9049
:10214000DF90CF900895EF92FF920F931F93CF935C
:10215000DF937B018C01E901E5EAF2E020E0808178
:102160009181A281B3818E159F05A007B10711F45B
:10217000922F0DC02F5F3D96243089F7CD2BF9F0BB
:102180009091D902892F8F5F83708093D9028DE05F
:10219000989FF0011124EB55FD4FEF012496DA01D1
:1021A00086E00D9009928150E1F7E082F18202838E
:1021B000138380EB94E09387828781E08487CDB797
:1021C000DEB7E6E00C94193EACE1B0E0EAEEF0E1F7
:1021D0000C94F73DCE0101966CE170E00E94350948
:1021E0008F8198850E94262D4C016F857889898979
:1021F0009A890E942A2D5B016C01698D7A8D8B8DE5
:102200009C8D0E942A2D7B018C0189819A810E94DC
:10221000262D019709F071C08B819C810E94262D8B
:102220008050984009F069C08091DA029091DB02F9
:10223000A091DC02B091DD02E816F9060A071B073F
:1022400009F05BC0CE01439660E071E046E050E0EB
:102250000E94A73E009709F050C0AE14BF04C0060C
:10226000D10611F482E04AC08E01075F1F4FC601FC
:10227000B501A80121E030E00E94A31081E088169A
:102280009104D9F58CE190E090937E0280937D02D9
:102290008EE090E00E941E0A81E090E00E945909C1
:1022A00080E098E00E94590986E00E944C0984E091
:1022B0000E944C0982E090E00E94590980E091E080
:1022C00066E070E00E9483096091DA027091DB029F
:1022D0008091DC029091DD020E946A09C80166E0EB
:1022E00070E00E948309CE010F9664E070E00E94C6
:1022F000830986E098E00E94EC1180E06C96ECE0A7
:102300000C94133EEF92FF920F931F93E09085027F
:10231000F090860200918702109188022091DE02DF
:102320003091DF024091E0025091E102DA01C901EF
:102330008E299F29A02BB12B8F5F9F4FAF4FBF4F8F
:1023400049F48FE792E06FEF70E046E050E00E94C2
:10235000853E35C08091DA029091DB02A091DC02CB
:10236000B091DD028E259F25A027B12782239323DC
:10237000A423B5230097A105B10511F421E009C0FC
:10238000E090E202F090E3020091E4021091E50295
:1023900022E0E5EAF2E08485813099F48081918140
:1023A000A281B3818E159F05A007B10751F4AFE755
:1023B000B2E0349686E001900D928150E1F720E082
:1023C00005C03D9682E0E93DF80729F7822F1F916D
:1023D0000F91FF90EF9008950F931F938C018091C0
:1023E0007D0290917E020E9690937E0280937D02F4
:1023F00080E090E00E941E0A8FE792E066E070E0C5
:102400000E94830980E091E066E070E00E94830909
:10241000C8010E94590988ED99E10E94540A1F9150
:102420000F910895AEE0B0E0E8E1F2E10C94003ED7
:10243000CE0101960E94C70C8823F1F0AFE7B2E00D
:10244000FE01379686E001900D928150E1F78D856F
:102450009E850E94262D28E08030920711F411E01D
:102460000CC08650984031F40E94E410182F0E944E
:10247000380A03C00E94380A10E0812F2E96E3E04C
:102480000C941C3EA8E0B0E0E8E4F2E10C94FF3DBF
:1024900060917D0270917E0282E290E00E94480B82
:1024A000892B11F087E065C082E290E00E94F90973
:1024B000CE01019668E070E00E9435099981909301
:1024C000E9028A818093EA02983031F16D817E8140
:1024D0008F8198850E942A2D9B01AC016093EB02AD
:1024E0007093EC028093ED029093EE028091E902EA
:1024F000833019F40E94170C3BC08530C9F58091D8
:10250000EA028130A9F52093E2023093E30240937E
:10251000E4025093E5022CC040917D0250917E026E
:1025200082E290E062E270E00E94720B82E290E050
:102530000E941E0A80E00E944C0980E00E944C0923
:1025400080E090E00E94590960917D0270917E02C6
:1025500082E290E00E94570B8C0184E290E00E949E
:102560001E0AC8010E94590981E00E94171301C088
:102570008AE02896E4E00C941B3EA0E0B0E0E3EC97
:10258000F2E10C94FA3DB82EEB016A01E9E9F2E0C0
:10259000EE24FF248701308121813296C901A0E019
:1025A000B0E0E80EF91E0A1F1B1F82E0E53AF807AB
:1025B00091F781E0B81651F480E00E94B108C7524B
:1025C000D64E80E0BE010E948B0803C0CE010E945F
:1025D000F909C6010E94F20A9C0140E050E02E0D6C
:1025E0003F1D401F511F203080E0380781E0480721
:1025F00080E05807A0F0CA0140E050E0A0E0B0E061
:10260000280F391F4A1F5B1F203080E0380781E008
:10261000480780E0580718F0C90101969C012095F1
:102620003095C901CDB7DEB7E9E00C94163EACE1B8
:10263000B0E0EDE1F3E10C94FF3D182F80917D02B5
:1026400090917E02449690937E0280937D028EE06C
:1026500090E00E941E0A80E095E40E945909809152
:102660007D0290917E020E9459098091E60290912C
:10267000E7020E94590980E090E40E94590980E431
:102680000E944C09812F0E944C0980E090E00E943A
:1026900059096091DA027091DB028091DC0290911D
:1026A000DD020E946A096091850270918602809124
:1026B0008702909188020E946A098EE090E064E1AE
:1026C00070E00E94570B8C0188E190E00E941E0A86
:1026D000C8010E9459090E948211882309F443C04D
:1026E000DE011196EDE7F2E09CE101900D92915030
:1026F000E1F7823049F46091E2027091E302809147
:10270000E4029091E50208C0609185027091860212
:1027100080918702909188020E9448100E94380A96
:102720000E943E0E8C01A8950E941212882311F07F
:102730000E94380A0E948211882311F420E008C008
:102740000E943E0E801B910B8C52914060F326E05C
:10275000ADE7B2E0FE0131968CE101900D9281501F
:10276000E1F7222329F480E098E00E94EC1120E0B8
:102770008091E6029091E70201969093E7028093A0
:10278000E602822F6C96E4E00C941B3EA4E1B0E0DC
:10279000ECECF3E10C94FD3D0E941212882309F445
:1027A000A1C0823011F485E09DC08EE090E064E12C
:1027B00070E00E94480B892B09F091C08EE090E0F8
:1027C0000E94F909CE01019664E170E00E9435098A
:1027D00069897A898B899C890E942A2D7B018C01C9
:1027E0002091DE023091DF024091E0025091E1023F
:1027F0008981682F70E0CB01807F907080349105D3
:1028000009F06DC08091DA029091DB02A091DC02A8
:10281000B091DD02E816F9060A071B0799F02E2988
:102820003F29402B512B2F5F3F4F4F4F5F4F51F0B0
:102830008FEFE8168FEFF8068FEF08078FEF180776
:1028400009F04DC06F707070660F771F660F771FAD
:102850006093E8028B819C810E94262D2091E802E2
:10286000821B910990937E0280937D026D857E8507
:102870008F8598890E942A2D609385027093860225
:102880008093870290938802E0928902F0928A02F4
:1028900000938B0210938C028091E802853120F026
:1028A000845190E00E94E30B609185027091860252
:1028B00080918702909188024FE752E020E030E05B
:1028C0000E94A3108A85813011F482E00BC081310F
:1028D00011F483E007C0863011F484E003C00E9445
:1028E000380A80E06496E6E00C94193EA0E0B0E07F
:1028F000ECE7F4E10C94FC3DD82EEB017A0184E185
:1029000090E0E80EF91EF0927E02E0927D028CEEDD
:102910009FEFE80EF91E82E290E00E941E0A8D8170
:102920009E810E9459098F8198850E945909698565
:102930007A858B859C850E946A096D857E858F8549
:1029400098890E946A0980E50E944C098D2D8F7339
:102950000E944C0984EB95E00E94590960E070E008
:1029600080E090E00E946A096091DA027091DB02D7
:102970008091DC029091DD020E942A2D60939902E1
:1029800070939A0280939B0290939C0269817A8152
:102990008B819C810E942A2D60939D0270939E02E0
:1029A00080939F029093A0021092A10286E08093F0
:1029B000A20280917D0290917E020E94262D90932A
:1029C000A4028093A30240917D0250917E0281E097
:1029D00062E270E00E94BD128C0182E390E00E94EE
:1029E0001E0AC8010E94590986E00E941713682F29
:1029F000882311F58D2D992787FD90958370907010
:102A0000892B41F089859A85AB85BC850196A11DEE
:102A1000B11D0EC0E114F10479F0970140E050E0DF
:102A200089859A85AB85BC85820F931FA41FB51F2E
:102A300089879A87AB87BC87862FCDB7DEB7E7E05B
:102A40000C94183EA2E1B0E0E8E2F5E10C94013EFE
:102A500020918D0230918E02C901A0E0B0E08A83FE
:102A60009B83AC83BD8380918F02909190029F8362
:102A70008E83398728871A861B861C861D8680913F
:102A8000950290919602A0919702B09198020196BA
:102A9000A11DB11D8E879F87A88BB98B84E0BE01D5
:102AA0006F5F7F4F40E050E00E9476146296E2E054
:102AB0000C941D3EA8E0B0E0E0E6F5E10C94F73D93
:102AC0007C0180919102909192020E94F90900E0AC
:102AD00010E06E010894C11CD11C2BE1A22E24E051
:102AE000B22EAE0CBF1C92E0892E9924939453C051
:102AF000C60165E070E04AE00E94C80B080F191F8C
:102B0000C60165E770E00E94443E892B91F4E11410
:102B1000F10419F087E993E002C087E193E06BE7E5
:102B200070E04AE00E94C80B080F191FF50190825F
:102B300032C0C60160E770E044E050E00E945D3EB4
:102B4000892B19F4F501808226C089818D30E1F44A
:102B50008A818A30C9F48091930290919402081777
:102B60001907C8F0EE0CFF1C87E194E0E80EF91E8F
:102B700081E090E0F7019183808315C00F5F1F4FC4
:102B80000E94FA088A3039F0809193029091940261
:102B90000817190798F380919302909194020817EF
:102BA000190708F4A5CF2896ECE00C94133ECF93B8
:102BB000DF93EC01009719F027E933E002C027E129
:102BC00033E0FE01EE0FFF1FDF0143E0AA0FBB1F42
:102BD0004A95E1F7AE0FBF1FA151BD4F1C92119650
:102BE0001D921D921D921C92149716961C921E9275
:102BF000159718961C921E9217971D961D921D925E
:102C00001D921C92509780E8D9011D928A95E9F790
:102C1000E95EFB4F11821082C55EDB4F1882DF91A7
:102C2000CF910895A6E2B0E0E8E1F6E10C94F33D1F
:102C30000091E80210E0025F1F4FCE01439664E16D
:102C400070E00E9435098B899C890E94262D909303
:102C50008E0280938D028D899E890E94262D9093ED
:102C6000900280938F026F89788D898D9A8D0E9452
:102C70002A2D609395027093960280939702909309
:102C800098022F8D2695269530E0C801820F931F5C
:102C9000909392028093910280917D0290917E02A6
:102CA000821B930B90939402809393026091850210
:102CB0007091860280918702909188020E942A2D4D
:102CC0006093990270939A0280939B0290939C0266
:102CD0006091890270918A0280918B0290918C029E
:102CE0000E942A2D60939D0270939E0280939F0202
:102CF0009093A0021092A10286E08093A20280919C
:102D00007D0290917E020E94262D9093A4028093D2
:102D1000A30240917D0250917E0280E0B8010E94A2
:102D2000BD12892B09F099C198A1992309F495C185
:102D30006090850270908602809087029090880251
:102D4000E0908D02F0908E02A0908F02B0909002E1
:102D50000FEE12E0CC24DD246FEF7FEF2E010894FC
:102D6000411C511CD201F80182E101900D92815069
:102D7000E1F7AE81BF81E885F9852A813B814C81ED
:102D80005D818981882331F48FEF6F3F780711F4DB
:102D9000B6010BC0261537054805590531F4EE1567
:102DA000FF0519F4AA15BB05C1F00894C11CD11C7C
:102DB0000E5E1F4FE2E0CE16D104A1F6FFEF6F3F8B
:102DC0007F0741F06B01C094D0948CE9C8168FEF57
:102DD000D80619F40E942215FFC0D7FE47C091FF04
:102DE0003FC18091130390911403A816B90609F00E
:102DF00037C1C094D094C601880F991F8C0143E05D
:102E0000000F111F4A95E1F7080F191F01511D4FBF
:102E1000F8016182728283829482B682A582F086F2
:102E2000E78281E080830E94B52CF8016187728778
:102E3000838794878091950290919602A091970242
:102E4000B09198020196A11DB11D85879687A7872D
:102E5000B08B8CE3818B82E1B80140E050E00E94AE
:102E60007614F82E882309F4FCC053C091FF03C0E8
:102E70000E9422154DC092FF0FC0B601660F771F4A
:102E8000CB0123E0880F991F2A95E1F7680F791F7E
:102E900061517D4F84E038C090FF3FC0C601880F6C
:102EA000991F8C01B3E0000F111FBA95E1F7080FCD
:102EB000191F01511D4FF8012081809195029091B9
:102EC0009602A0919702B09198020196A11DB11DA2
:102ED00085879687A787B08B223079F480E1B80187
:102EE00040E050E00E94761481E1B80140E050E0FB
:102EF0000E947614F82E85E0A1C0233019F0263008
:102F000009F0AEC080E1B80140E050E00E947614C4
:102F1000F82EC6010E94D715A4C093FF5FC0809110
:102F2000930290919402009711F480E055C05601ED
:102F3000AA0CBB1C8501F3E0000F111FFA95E1F705
:102F40000A0D1B1D01511D4FF8012081213019F47C
:102F500082E0808302C0223011F0FF243CC0A0E058
:102F6000B0E02091950230919602409197025091E5
:102F70009802820F931FA41FB51FF80185879687BB
:102F8000A787B08B2581368180911303909114031C
:102F900028173907B1F480E1B80140E050E00E9401
:102FA0007614F82EC6010E945A15F501E95EFB4F12
:102FB00080819181019779F4C6010E94482FF82EF3
:102FC0000AC081E1B80140E050E00E947614F82E7A
:102FD00083E0F80180838F2DF82E43C094FF40C01A
:102FE000C601880F991F8C0173E0000F111F7A959D
:102FF000E1F7080F191F01511D4FF8018081813041
:1030000011F482E022C08230E1F480919302909129
:103010009402892B59F080E1B80140E050E00E9411
:103020007614F82EC6010E945A151BC081E1B80122
:1030300040E050E00E947614F82E83E0F80180838F
:1030400010C0833021F486E0F801808309C0853008
:1030500039F4C6010E94D71503C068E0F62E01C0FE
:10306000FF248F2DA696E0E10C940F3ECF93DF93C3
:10307000089690937E0280937D0282E290E00E9407
:103080001E0A80918F02909190020E9459098091AE
:103090008D0290918E020E94590980917D0290913B
:1030A0007E020E94590980E090E00E9459096091D7
:1030B000DA027091DB028091DC029091DD020E94C5
:1030C0002A2D6093990270939A0280939B029093A9
:1030D0009C02609185027091860280918702909196
:1030E00088020E942A2D60939D0270939E02809315
:1030F0009F029093A0021092A10281E18093A2020C
:1031000080917D0290917E020E94262D9093A402D0
:103110008093A30240917D0250917E0281E062E2A1
:1031200070E00E94BD12EC01009711F4CFEFDFEFC9
:1031300088E290E00E941E0ACE010E94590981E1B6
:103140000E941713DF91CF910895A8E0B0E0EBEA59
:10315000F8E10C94FD3DCE01019668E070E00E941C
:10316000350989819A810E94262D90938E02809341
:103170008D028B819C810E94262D909390028093DA
:103180008F028D819E810E94262D7C0188EF9FEF0A
:10319000E80EF91EF0929402E092930288E090E02B
:1031A000E80EF91E8091E802082F10E0025F1F4F21
:1031B0008F819885892BC1F160918502709186027B
:1031C00080918702909188020E942A2D6093990233
:1031D00070939A0280939B0290939C026091890263
:1031E00070918A0280918B0290918C020E942A2D0C
:1031F00060939D0270939E0280939F029093A00221
:103200001092A10281E18093A2028D819E81909310
:10321000A4028093A30280E0B801A7010E94BD121E
:10322000892B11F089E024C0085F1F4F1093920290
:103230000093910280918F02909190028B379105BB
:1032400019F40E94952414C024E08030920719F4E8
:103250000E94D81E0DC08434910519F40E949E1C52
:1032600007C08938910511F080E002C00E9420203B
:103270002896E6E00C94193E809193049091940472
:10328000A0919504B0919604809385029093860254
:10329000A0938702B093880283E490E090938E021B
:1032A00080938D0284E490E09093900280938F024B
:1032B0008AE290E00E941E0A60E076E081E091E000
:1032C0000E946A090E94B52C6093A7047093A80419
:1032D0008093A9049093AA040E946A0980E090E078
:1032E0000E94590980E090E00E94590960E070E076
:1032F00080E090E00E946A0980E06CE070E00E944B
:103300009B0980E091E066E070E00E94830980E024
:103310006AEC70E00E949B0963E673E582E893E63D
:103320000E946A0981E095E30E94590984E00E94A5
:103330004C0982E30E944C0984E00E944C09609190
:10334000DA027091DB028091DC029091DD020E9432
:103350006A0986E30E944C0984E00E944C0960914E
:1033600093047091940480919504909196040E9426
:103370006A098FEF0E944C0980E06CE270E00E94C5
:103380009B098CE291E00E94361808950F931F93D9
:1033900081E08093BE048FEF9FEFAFEFBFEF80938C
:1033A000850290938602A0938702B093880283E4FB
:1033B00090E090938E0280938D0284E490E090934D
:1033C000900280938F021092DE021092DF02109220
:1033D000E0021092E1021092DA021092DB021092E7
:1033E000DC021092DD021092A3051092A405109247
:1033F000A5051092A6051092E2021092E302109227
:10340000E4021092E50210928F0410929004109240
:1034100091041092920410928B0410928C041092DA
:103420008D0410928E0410929704109298041092BA
:10343000990410929A04109293041092940410929A
:103440009504109296041092A3041092A404109272
:10345000A5041092A60410929B0410929C04109252
:103460009D0410929E0410929F041092A00410924A
:10347000A1041092A2041092B3041092B40410920A
:10348000B5041092B6041092C1040E94B52C60934A
:10349000A7047093A8048093A9049093AA048AE2D5
:1034A00090E00E941E0A60E076E081E091E00E94D8
:1034B0006A096091A7047091A8048091A904909171
:1034C000AA040E946A0960E070E880E090E00E942F
:1034D0006A0980E060E170E00E949B0900E011E071
:1034E000C80166E070E00E94830980E06AEC70E049
:1034F0000E949B0963E673E582E893E60E946A09ED
:1035000081E095E30E94590981E00E944C098DE316
:103510000E944C0987E00E944C0981E00E944C09FE
:10352000C80166E070E00E9483098FEF0E944C0999
:1035300080E06FE270E00E949B098CE291E00E94C3
:1035400036181F910F9108950F931F93182F809392
:10355000BE04883129F08FEF9FEFAFEFBFEF08C0B7
:103560008091930490919404A0919504B091960455
:103570008093850290938602A0938702B09388027D
:10358000133051F00E94B52C6093A7047093A804E7
:103590008093A9049093AA04E3E9F5E00190002048
:1035A000E9F73197E359F5400E2F0F5F83E490E080
:1035B00090938E0280938D0284E490E09093900229
:1035C00080938F028AE290E00E941E0A60E076E01B
:1035D00081E091E00E946A096091A7047091A804BB
:1035E0008091A9049091AA040E946A0980E090E069
:1035F0000E945909183119F080E090E802C080E07B
:1036000090E00E9459096091DA027091DB0280918A
:10361000DC029091DD020E946A0980E06CE070E0BB
:103620000E949B0980E091E066E070E00E948309BF
:1036300080E06AEC70E00E949B0963E673E582E833
:1036400093E60E946A0981E095E30E94590983E0AC
:103650000E944C098CE00E944C09802F0E944C096A
:1036600083E995E0602F70E00E948309133019F51B
:1036700082E30E944C0984E00E944C0980919102EF
:103680009091920240960E94F9090E9419090E94A5
:103690006A0986E30E944C0984E00E944C0960910B
:1036A00093047091940480919504909196040E94E3
:1036B0006A0919E115C0163111F015E211C082E353
:1036C0000E944C0984E00E944C096091870470912B
:1036D00088048091890490918A040E946A091FE1FC
:1036E00087E30E944C0986E00E944C0981E00E9419
:1036F0004C0983E00E944C0986E00E944C0983E358
:103700000E944C098AE30E944C098BE30E944C09F9
:103710008DE30E944C0987E00E944C0981E00E94E1
:103720004C0980E091E066E070E00E9483098FEF31
:103730000E944C09101B80E0612F70E00E949B09E1
:103740008CE291E00E9436181F910F910895EF923C
:10375000FF920F931F938091BF049091C004892B17
:1037600059F4ABE0B1E0EFE1F1E082E101900D92BC
:103770008150E1F760E0DCC08091BE04813031F01F
:10378000863121F0883111F08931D9F5E090BB0400
:10379000F090BC0400E010E08BE091E06FE171E09C
:1037A0000E94C32DE61AF70A080B190BE092B70422
:1037B000F092B8040093B9041093BA041E141F04C5
:1037C00010061106F4F08091BE04813049F0863174
:1037D00059F48091C1048F5F8093C104833018F045
:1037E0000E94C61903C086E10E94A41A682FABE0AC
:1037F000B1E0EFE1F1E082E101900D928150E1F75B
:1038000001C060E0E090B304F090B4040091B5040E
:103810001091B604D801C7010196A11DB11D0297F0
:10382000A105B10508F484C08091AB049091AC046B
:10383000A091AD04B091AE042091AF043091B004DA
:103840004091B1045091B2040097A105B10591F1E6
:103850000197A109B1098093AB049093AC04A093A4
:10386000AD04B093AE04215030404040504020930E
:10387000AF043093B0044093B1045093B204089461
:10388000E108F10801091109E092B304F092B404CF
:103890000093B5041093B6040097A105B10509F093
:1038A00047C088E10E94A41A682F882309F040C00D
:1038B0006CE03EC00894E108F108010911092115E6
:1038C00031054105510509F1DA01C9010197A10945
:1038D000B1098093AF049093B004A093B104B09366
:1038E000B204E092B304F092B4040093B5041093D0
:1038F000B6040097A105B105D9F489E10E94A41A84
:10390000682F8823A9F46DE013C0E092B304F0920D
:10391000B4040093B5041093B604E114F104010556
:10392000110531F40E94C619682F882309F46EE04E
:10393000862F1F910F91FF90EF900895ACE1B0E0BA
:10394000E4EAFCE10C94FD3D8091BE04882309F477
:10395000E2C1873109F4DFC1809191029091920216
:1039600080519F4F0E94F9090E94FA08182F8F3F3B
:1039700009F4C5C00E94FA08082F153341F48130BC
:1039800009F0D0C10E94FA088093BD04EDCF113038
:1039900071F4843009F0C6C10E94190960938B0448
:1039A00070938C0480938D0490938E04DDCF13303C
:1039B00071F4843008F4B6C10E94190960938F0431
:1039C0007093900480939104909392041FC01633D7
:1039D00071F4843008F4A6C10E941909609393041D
:1039E0007093940480939504909396040FC01630BE
:1039F000A1F4843008F496C10E94190960939704D9
:103A0000709398048093990490939A04043009F475
:103A1000ABCF802F90E004976FC0133309F04BC0F9
:103A2000843009F0A1CF0E9419097B018C016093B9
:103A3000A3047093A4048093A5049093A60480919A
:103A40009F049091A004A091A104B091A2040097BA
:103A5000A105B105B1F4C801B7012BE633E040E0A0
:103A600050E00E94753D28EE33E040E050E00E94B7
:103A7000B43D20939F043093A0044093A10450933D
:103A8000A20480919B0490919C04A0919D04B0910C
:103A90009E040097A105B10509F066CF169507951C
:103AA000F794E794E0929B04F0929C0400939D04A9
:103AB00010939E0459CF1A3371F4843009F054CF17
:103AC0000E94190960939B0470939C0480939D0449
:103AD00090939E0449CF1B3371F4843009F044CF96
:103AE0000E94190960939F047093A0048093A1041D
:103AF0009093A20439CF90E00E94E30B35CF8091E0
:103B000091029091920204960E94F9098091BE045C
:103B10009091BD048130B9F4923009F0FEC00E944A
:103B200019092091A7043091A8044091A90450914B
:103B3000AA04621773078407950709F0EEC083E0B3
:103B40000E94A41AEBC0953009F0D3C00E94190955
:103B50002091A7043091A8044091A9045091AA048F
:103B6000621773078407950709F0D7C087E1809330
:103B7000BE04809191029091920240960E94F909B0
:103B80000E941909AB01BC014093DA025093DB0299
:103B90006093DC027093DD0288E090E00E940A3FAF
:103BA00080918B0490918C04A0918D04B0918E042F
:103BB0008093DE029093DF02A093E002B093E102D3
:103BC00080918F0490919004A0919104B0919204FF
:103BD0008093E2029093E302A093E402B093E502A3
:103BE0008091970490919804A0919904B0919A04BF
:103BF0008093A3059093A405A093A505B093A60573
:103C000080919B0490919C04A0919D04B0919E048E
:103C10008093AB049093AC04A093AD04B093AE0436
:103C200080919F049091A004A091A104B091A2045E
:103C30008093AF049093B004A093B104B093B20406
:103C40008091A3049091A404A091A504B091A6042E
:103C50008093B3049093B404A093B504B093B604D6
:103C60008F5F9F4FAF4FBF4F21F41092C00410924F
:103C7000BF04DE011196EDE7F2E08CE101900D92B8
:103C80008150E1F76091DA027091DB028091DC02F1
:103C90009091DD020E9448100E94380A0E943E0E58
:103CA0008C01A8950E941212813019F40E94380AE2
:103CB00009C0823039F40E943C19882381F40E94A3
:103CC000C6190DC00E943E0E801B910B4E9748F303
:103CD00081E090E09093AA058093A90580E0ADE78C
:103CE000B2E0FE0131969CE101900D929150E1F716
:103CF00015C0963091F40E9419092091A7043091C3
:103D0000A8044091A9045091AA046217730784077C
:103D1000950719F407C080E001C08FE06C96E6E0DB
:103D20000C94193E0E94C619F9CFAF92BF92DF9250
:103D3000EF92FF920F931F93DF93CF930F92CDB724
:103D4000DEB7F82EE92E9C0159018EE2D82E0E9492
:103D5000FA08982F882331F40894A108B108F501D6
:103D6000108219C0807C803C11F085010AC00E943D
:103D7000FA0811C099830E94FA08F80181938F0113
:103D80009981802F8A198917A8F3A90EB11CF50112
:103D9000D1925F01DCCF8F2D9E2D0F90CF91DF91BF
:103DA0001F910F91FF90EF90DF90BF90AF9008951B
:103DB000ACE4B0E0EEEDFEE10C94F33D80919102B5
:103DC000909192020E94F909CE0101966CE070E098
:103DD0000E94350989819A810E94262D20918805AB
:103DE000309189058217930709F06AC08D819E8101
:103DF0000E94262D6C01EE24FF243DE2A32EB12C5F
:103E0000AC0EBD1E2DE0822E912C8C0E9D1E14C07A
:103E1000C5010E94951E0E9407098C010E94070996
:103E20000130110531F4019721F4C401B5010E945C
:103E3000A03E0894E11CF11CEC14FD0448F38F81B2
:103E400098850E94262D3C01EE24FF249DE2492EF8
:103E5000512C4C0E5D1E31C0C2010E94951E0E9465
:103E600007098C010E9407094C010E9419095B0196
:103E70006C010E94070901301105D1F421E082167E
:103E80009104B1F48430910599F40E941909AB01B1
:103E9000BC0140938A0550938B0560938C05709309
:103EA0008D05CE010D96960185010E94FE2208C067
:103EB0000E94E30B0894E11CF11CE614F70460F285
:103EC00080E0C45BDF4FE0E10C940F3EAF92BF9205
:103ED000DF92EF92FF920F931F93CF93DF93182FF0
:103EE000092F8091A3059091A405A091A505B091FB
:103EF000A6058093850290938602A0938702B093D3
:103F0000880285E390E090938E0280938D0280E09A
:103F100094E09093900280938F020E94B52C70934E
:103F20008905609388058AE290E00E941E0A8091CC
:103F30008805909189050E94590980E091E00E94CE
:103F4000590981E090E00E94590980E090E00E94C8
:103F5000590980E090E00E94590980E090E00E94B9
:103F60005909212F302FC901EC0140E1A42EB12CB9
:103F70007E010E2D0C1BF701D080FEE2DF1631F022
:103F8000DD2021F00894E11CF11CF3CF802F0E946A
:103F90004C0910E0CE01B8010E9483090F5F1F4F4A
:103FA000A00EB11EDD2019F0E7012196E1CF80E0DF
:103FB0000E944C0981E090E00E94590981E090E064
:103FC0000E945909C50101960E943618DF91CF91D0
:103FD0001F910F91FF90EF90DF90BF90AF900895E9
:103FE0001F930E94FA08182F11541295107F0E94F7
:103FF000FA0881548F70812B1F9108950F931F939E
:10400000CF93DF93EC0100E0899190E00E943C3E69
:10401000182F85958595859585958F5B0E944C0910
:104020001F70812F8F5B0E944C090F5F003161F779
:1040300080E00E944C09DF91CF911F910F9108956C
:10404000ACE1B0E0E6E2F0E20C94F33D8091910245
:10405000909192020E94F909CE0101966CE070E005
:104060000E9435098B819C810E94262D9C018F70B6
:104070009070892B11F082E1EEC037FF5AC0898120
:104080009A810E94262D20918805309189058217FA
:10409000930709F0DFC08F8198850E94262D019734
:1040A00011F080E1D8C00E94FA08803211F081E15D
:1040B000D2C08E01035F1F4FC801902E892E2DE1C3
:1040C000E22EF12CEC0EFD1E0E94F01FF8018193F0
:1040D0008F01EE15FF05C1F71C8E0E94FA080E94A1
:1040E00007098C010E9407097C010E9419095B01E4
:1040F0006C010032110509F0ADC0F1E0EF16F104DA
:1041000009F0A8C00E9407090E9407090E94190926
:10411000AB01BC0140938A0550938B0560938C05DD
:1041200070938D05892D982D960185010E94FE22A0
:1041300091C020703877232B09F08CC080919302B6
:1041400090919402C29709F085C089819A810E945A
:10415000262D4C018D819E810E94262D5C01CC2450
:10416000DD249DE0692E712C6C0E7D1E8DE1482EA4
:10417000512C4C0E5D1E31C00E94FA08803209F0AD
:1041800069C083010E94F01FF80181938F01E4153B
:10419000F505C1F71C8E0E94FA080E9407097C01F0
:1041A0000E9407090197B1F4F0E2EF16F10451F40F
:1041B000C30163E975E00E94973E009759F400E05F
:1041C00015E84FC081E2E816F10421F48D858A32AA
:1041D00009F445C00894C11CD11CCA14DB0460F268
:1041E00039C086E090E00E94590980E090E00E948A
:1041F00059096091DA027091DB028091DC029091A2
:10420000DD020E946A098EE390E021C08DE390E018
:104210000E94590981E00E944C0983E995E06FE012
:1042200070E00E94830980E00E944C0980E094E0E5
:104230000E94590980E091E066E070E00E948309E5
:1042400080E064E270E00E949B0985E790E00E94B4
:10425000361801C080E06C96E0E10C940F3E00E05F
:1042600014E88AE290E00E941E0AC4010E945909E3
:10427000C8010E94590980E090E00E94590981E03C
:1042800090E00E94590980E090E00E94590980E086
:1042900090E00E94590980E20E944C09CE010D96DF
:1042A0000E94FE1FC7010E94590981E090E00E9410
:1042B000590968E572E080E090E00E946A09E0E256
:1042C000EE16F10409F0A2CF8CCF0F931F938C014F
:1042D0008091DE029091DF02A091E002B091E102B4
:1042E00080959095A095B0952091DA023091DB02EF
:1042F0004091DC025091DD02822B932BA42BB52B35
:104300008093850290938602A0938702B0938802DF
:1043100089E890E090938E0280938D0290939002B2
:1043200080938F020E94B52C709389056093880555
:104330008AE290E00E941E0A80918805909189058A
:104340000E94590980E191E00E94590981E090E0C2
:104350000E94590980E090E00E94590980E090E0B5
:104360000E94590980E090E00E94590980E20E9471
:104370004C09C8010E94FE1F80E290E00E9459098A
:1043800081E090E00E94590982E390E00E94361893
:104390001F910F910895E6E0F5E084818130A1F44A
:1043A00080819181A281B3810097A105B10561F05F
:1043B0000197A109B10980839183A283B3830097F8
:1043C000A105B10509F41482B99685E0EA3AF80727
:1043D00021F70895A9E2B0E0E0EFF1E20C94FB3D93
:1043E0007C0102EE14E06E010894C11CD11CD601C0
:1043F000F80189E201900D928150E1F789A58130A1
:1044000059F4C601B7010E94973E009729F429A1EB
:104410003AA14BA15CA10AC0075D1F4F85E0063899
:10442000180729F720E030E040E050E0B901CA0168
:10443000A996E8E00C94173ECF93DF938091900506
:10444000813001F5C2ECD4E0CE016AE875E00E944B
:10445000302D813009F4C3C0FE0101900020E9F73E
:104460003197EC1BFD0B709738F4CE016EE270E0D3
:104470000E948C3E009711F084E001C082E080939E
:104480009005A9C0823009F582EC94E00E94EA21EF
:1044900060938A0570938B0580938C0590938D05AE
:1044A000611571058105910509F099C00E943E0EC4
:1044B000909387058093860582EC94E00E946521A5
:1044C000282F10928F0583E053C0833079F58091B7
:1044D0008A0590918B05A0918C05B0918D05009770
:1044E000A105B10509F07BC00E943E0E2091860512
:1044F00030918705821B930B8C52914008F46BC05E
:1045000080918F058F5F80938F05833020F02091FD
:1045100061042D5E61C00E943E0E909387058093DA
:10452000860582EC94E00E94652153C0843019F521
:1045300082EC94E00E94EA2160938A0570938B05D7
:1045400080938C0590938D0561157105810591050A
:1045500009F045C00E943E0E909387058093860522
:1045600082EC94E00E94661F282F10928F0585E050
:104570008093900531C0853071F580918A059091C6
:104580008B05A0918C05B0918D050097A105B10513
:1045900031F50E943E0E2091860530918705821BE1
:1045A000930B8C529140B8F080918F058F5F809370
:1045B0008F05833020F020916104295E0DC00E9498
:1045C0003E0E909387058093860582EC94E00E94CE
:1045D000661F282F01C020E080E090E003C020E0AB
:1045E00081E090E09093920580939105019711F4FA
:1045F00010929005822FDF91CF910895A0E0B0E056
:10460000E4E0F3E20C94F73DEC016A017B01480120
:10461000590182EE94E0BE010E94973E0097B9F1E5
:104620008BE095E0BE010E94973E009781F184E304
:1046300095E0BE010E94973E009749F18DE595E017
:10464000BE010E94973E009711F120918E05822FA6
:104650008F5F837080938E0530E089E290E0289F21
:104660008001299F100D389F100D11240E511B4FF2
:10467000C801BE010E94A03EF801C0A2D1A2E2A2E0
:10468000F3A284A295A2A6A2B7A281E080A7CDB78B
:10469000DEB7ECE00C94133EA8E0B0E0E2E5F3E214
:1046A0000C94F93D6D837E838F83988719821A82DB
:1046B0001B821C8229813A814B815C81ECE2AE2E07
:1046C000BB24B394CC24DD24EE24FF2400E010E0CE
:1046D0000E940037952FB901842F2896EAE00C94A8
:1046E000153EA0E2B0E0E7E7F3E20C94FD3D7C016B
:1046F000E62FF0E0EE0FFF1FE155FF4F659174913B
:104700008E010F5F1F4FC8010E94A03EC801B70174
:104710000E94302DA096E6E00C94193EEF92FF9295
:104720001F93DF93CF9300D000D0CDB7DEB7809139
:10473000610480936204182F1F5F11707E0108943A
:10474000E11CF11CC701612F0E9471238130C1F46B
:1047500089819A81AB81BC810097A105B10581F463
:104760001F5F1170C701612F0E947123813041F4D6
:1047700089819A81AB81BC810097A105B10511F0B7
:10478000109361040F900F900F900F90CF91DF91D5
:104790001F91FF90EF900895AF92BF92CF92DF925A
:1047A000EF92FF920F931F9360938502709386029E
:1047B00080938702909388028BE790E090938E021B
:1047C00080938D029093900280938F028AE290E012
:1047D0000E941E0A83E20E944C0980E067E270E0BA
:1047E0000E949B09F894E090C305F090C4050091E5
:1047F000C5051091C6056091C1057091C205882755
:1048000077FD8095982F0E944C235B016C01789472
:1048100060936F047093700480937104909372049A
:1048200080E89EE7AAEAB3E8E80EF91E0A1F1B1FFC
:10483000C801B7010E946A09C601B5010E946A0950
:1048400080E390E00E9436181F910F91FF90EF9047
:10485000DF90CF90BF90AF9008951F931091B00557
:10486000112309F45EC01130A1F480916104E82F96
:10487000F0E0EE0FFF1FE155FF4F6591749182EC60
:1048800094E00E94A03E1093900582E08093B005D2
:1048900048C0123079F58091910590919205019769
:1048A00009F03FC0109292051092910560918A051F
:1048B00070918B0580918C0590918D0560931D04FE
:1048C00070931E0480931F04909320040E94CC23B5
:1048D000182F882351F483E08093B0050E943E0E88
:1048E0009093800480937F0402C01092B0050E94D0
:1048F0008E2318C01330A9F40E943E0E20917F042D
:1049000030918004821B930B2091810430918204AA
:104910008217930730F01093060110916204145E21
:1049200001C010E0812F1F910895A9E5B0E0EBE9E7
:10493000F4E20C94F13D80919102909192020E94D8
:10494000F909CE01819660E370E00E94350999A1D2
:10495000892F8770843009F0DAC38091B0058823ED
:1049600009F45CC7892F807C809307019AA1803C61
:1049700021F0992311F0903148F082E080930601F4
:10498000109290051092B0058BE149C79F5F9093FC
:1049900008016DA17EA18FA198A50E942A2D609388
:1049A0006704709368048093690490936A0469A50E
:1049B0007AA58BA59CA50E942A2D60936B04709309
:1049C0006C0480936D0490936E04FE01E05CFF4FD5
:1049D00090812FAD5EAD6DAD7CADABADDAAC99AC79
:1049E000FE01EC5BFF4FC080FE01ED5BFF4FB0802E
:1049F000FE01EE5BFF4FA080FE01EF5BFF4F70807A
:104A0000FE01E85BFF4F8081FE01E95BFF4F3081D3
:104A1000FE01EA5BFF4F4081FE01EB5BFF4FE0814F
:104A2000E82EE91A91E08E1508F090E0832F821BA2
:104A300021E0381708F020E0F82EF91A91E08F15E0
:104A400008F090E0292B842F851B31E0481708F0EF
:104A500030E0082F021B91E0801708F090E0392B1E
:104A60008E2F861B21E0E81708F020E0182F131B7B
:104A700091E0811708F090E0292B8C2D871B31E005
:104A8000C81608F030E0B82FB21B91E08B1708F081
:104A900090E0392B8B2D8A1B21E0B81608F020E01E
:104AA000A82FA31B91E08A1708F090E0292B8A2DEC
:104AB0008D1991E0A81608F090E0F82FF21B21E084
:104AC0008F1708F020E0922BE72DE919E91B9701D9
:104AD000A8016B2F7A2F8F2F9E2F52F52E2D2F5F2F
:104AE00081E02E1508F080E0382F3F0D81E03F1562
:104AF00008F080E0482F400F81E0401708F080E088
:104B0000582F510F81E0511708F080E0682F6B0F8C
:104B100081E06B1708F080E0782F7A0F81E07A1738
:104B200008F080E08F0F91E08F1708F090E09E0F63
:104B300001E00E947B36622E532E442E352E262E07
:104B400066967FAF669767968FAF679768969FAFB9
:104B50006897FE01E45BFF4FC080FE01E55BFF4FFD
:104B6000B080FE01E65BFF4FA080FE01E75BFF4FD8
:104B70007080FE01E05BFF4F0081FE01E15BFF4FB3
:104B8000F080FE01E25BFF4F9080FE01E35BFF4F90
:104B900080808091730490917404A0917504B09109
:104BA000760480589148A545BC47182F8D839E8375
:104BB000AF83B88760917B0470917C0480E090E0C3
:104BC0000E944C2369837A838B839C83872F3B814C
:104BD000492F5E817F81E885D02ED61A91E00D1590
:104BE00008F090E02F2D281B822F21E0F81608F006
:104BF00020E0E82EE91A91E08E1508F090E0292BCC
:104C0000892D831B31E0981608F030E0F82EF21A57
:104C100091E08F1508F090E0392B882D841B21E05E
:104C2000881608F020E0082F031B91E0801708F099
:104C300090E0292B3C2D311B132F91E0C31608F077
:104C400090E0B12FB21B81E01B1708F080E0982B99
:104C50008B2D851B21E0B81608F020E0A82FA91B9A
:104C600091E08A1708F090E0292B8A2D871B91E0AC
:104C7000A81608F090E0F82FF21B21E08F1708F03B
:104C800020E0922B7E1AE72DE91B2D2D3E2D4F2D76
:104C9000502F6B2F7A2F8F2F9E2F52F52D2D2F5F98
:104CA00081E02D1508F080E0382F3E0D81E03E15A3
:104CB00008F080E0482F4F0D81E04F1508F080E0AC
:104CC000582F500F81E0501708F080E0682F6B0FCD
:104CD00081E06B1708F080E0782F7A0F81E07A1777
:104CE00008F080E08F0F91E08F1708F090E09E0FA2
:104CF00001E00E947B36A32FB42F152F062FF72E2D
:104D0000D82EC22EC60CF1E0C21608F0F0E03A2F01
:104D1000350DE1E03A1708F0E0E0EF2EE30E21E078
:104D2000E31608F020E0E22B4B2F440D31E04B1747
:104D300008F030E0AE2FA40F21E0A41708F020E027
:104D4000322B512F530D41E0511708F040E0F32F63
:104D5000F50F21E0F51708F020E0422B602F620DDF
:104D600031E0601708F030E0E42FE60F21E0E617AD
:104D700008F020E0322B66967FAD66977F0D41E00C
:104D80007F1508F040E0532F570F21E0571708F028
:104D900020E0422B67968FAD67978D0D21E08D1532
:104DA00008F020E0480F31E0481708F030E0232BEE
:104DB00068968FAD6897980F290FC982EA82AB83F6
:104DC000FC83ED835E834F8328876D807E808F8098
:104DD0009884A980BA80CB80DC809501A60160E030
:104DE00070E080E090E002E00E94FC35122FF32E8C
:104DF000E42ED52EC62EA72E582E392E0E94FC3515
:104E0000B22EB10E21E0B11608F020E03F0DE1E036
:104E10003F1508F0E0E0422E430E21E0431608F073
:104E200020E0E22B4E0D31E04E1508F030E0EE2E82
:104E3000E40E21E0E41608F020E0322B5D0D41E0A5
:104E40005D1508F040E0D32ED50E21E0D51608F010
:104E500020E0422B6C0D31E06C1508F030E0C42EE0
:104E6000C60E21E0C61608F020E0322B7A0D41E094
:104E70007A1508F040E0A32EA70E21E0A71608F04F
:104E800020E0422B850D21E0851508F020E0542E0E
:104E9000580E31E0581608F030E0232BF32CF90EB1
:104EA000F20E2B2D342D4E2D5D2D6C2D7A2D852D52
:104EB0009F2D04E00E94FC35A32FB42F052F162F41
:104EC000372E282EE22FEB196996EFAF6997F1E0A4
:104ED0002E1708F0F0E03A2F3419E1E0A31708F09C
:104EE000E0E0B32EBF1A21E03B1508F020E0E22BF2
:104EF0004B2F4E1931E0B41708F030E0A42FAE1B51
:104F000021E04A1708F020E0322B502F5D1941E0D4
:104F1000051708F040E0F52FF31B21E05F1708F0BC
:104F200020E0422B612F6C1931E0161708F030E0B9
:104F3000E62FE41B21E06E1708F020E0322B732DE2
:104F40007A1941E0371608F040E0572F531B21E053
:104F5000751708F020E0422B822D851921E02816D4
:104F600008F020E0382F341B432F31E0841708F07D
:104F700030E0232B9F19921B69968FAD6997898723
:104F8000BA86AB87FC87ED875E874F87988BED8469
:104F9000FE840F85188980911D0190911E01892B37
:104FA00009F5609185047091860461157105D1F051
:104FB0008091B4059091B505892BA1F4A4019301CA
:104FC00097FE07C022273327A90126193709480968
:104FD0005909CB01A0E0B0E082179307A407B507F9
:104FE0000CF41CC497011092B5051092B405F89406
:104FF0008091C3059091C405A091C505B091C605E7
:10500000860D971DA81DB91D8093C3059093C405F7
:10501000A093C505B093C6058091C1059091C205C6
:105020008E0D9F1D9093C2058093C1058091C1058F
:105030009091C20597FF2AC08091C3059091C40545
:10504000A091C505B091C605181619061A061B06CB
:10505000ECF48091C3059091C405A091C505B09171
:10506000C6050197A109B1098093C3059093C405B2
:10507000A093C505B093C6058091C1059091C20566
:1050800088519C4F9093C2058093C1058091C305C0
:105090009091C405A091C505B091C6058093770491
:1050A00090937804A0937904B0937A048091C10519
:1050B0009091C20590937E0480937D04789497FE2E
:1050C0000AC0121613063CF40894611C711C811C62
:1050D000911C285E3340D401C30180509048AF4FEB
:1050E000BF4F80509040A140B04038F08FEF9FE715
:1050F000909364048093630404C07092640460928B
:105100006304309366042093650481E085C3833093
:1051100009F0F1C0292F28738091B2059091B30551
:105120000197F1F550900701522A40900801E09054
:105130007704F09078040091790410917A0480E863
:105140009EE7AAEAB3E8E80EF91E0A1F1B1F60914A
:105150007D0470917E0480E090E00E944C233B012E
:105160004C01A0907304B0907404C0907504D0906A
:10517000760480E89EE7AAEAB3E8A80EB91ECA1E24
:10518000DB1E60917B0470917C0480E090E00E94C3
:105190004C2365966CAF7DAF8EAF9FAF659713C004
:1051A00030EC532E522A65961CAE1DAE1EAE1FAEBD
:1051B0006597662477244301AA24BB246501EE2465
:1051C000FF24870144248AE290E00E941E0A852D74
:1051D00084600E944C09842D0E944C098BA10E947E
:1051E0004C0986EF0E944C0960E070E080E090E09E
:1051F0000E946A0960E070E080E090E00E946A0925
:105200006091DA027091DB028091DC029091DD0204
:105210000E946A09C801B7010E946A09C401B3016A
:105220000E946A098091B2059091B305019799F4A3
:10523000CE0181968C01085D1F4F20E3E22EF12CF8
:10524000E80EF91ED8018D918D010E944C090E15B2
:105250001F05C1F70CC060E070E080E090E00E94A4
:105260006A0960E070E080E090E00E946A09C6018F
:10527000B5010E946A0965966CAD7DAD8EAD9FAD9E
:1052800065970E946A098091B2059091B3050197D4
:1052900039F0AA24BB246501EE24FF2487011EC037
:1052A000F894E090C305F090C4050091C5051091F5
:1052B000C60580E89EE7AAEAB3E8E80EF91E0A1FD1
:1052C0001B1F6091C1057091C205882777FD8095ED
:1052D000982F0E944C235B016C017894C801B701A0
:1052E0000E946A09C601B5010E946A0980E390E044
:1052F0000E94361894C2853009F090C2892F807CB4
:10530000809307019AA1803C09F488C2992309F48B
:1053100085C2903108F082C29F5F909308016DA111
:105320007EA18FA198A50E942A2D60936704709397
:1053300068048093690490936A0469A57AA58BA593
:105340009CA50E942A2D60936B0470936C0480933B
:105350006D0490936E04FE01E05BFF4FD080FE0170
:10536000E15BFF4FC080FE01E25BFF4FA080FE01CA
:10537000E35BFF4F10813D2DD98A2C2DCA8A9A2DCF
:10538000AB8A812F1C8BFE01E45BFF4FD080FE01B6
:10539000E55BFF4FC080FE01E65BFF4FA080FE0192
:1053A000E75BFF4F1081DD8ACE8AAF8A188F032F0B
:1053B000F22EE92EB82E832F822B892B8B298D2953
:1053C0008C298A29812B09F429C2F8948091C3057C
:1053D0009091C405A091C505B091C605805891482B
:1053E000A545BC478D8B9E8BAF8BB88F6091C10557
:1053F0007091C205882777FD8095982F0E944C23D5
:10540000698B7A8B8B8B9C8B789489892A893B89D1
:105410004C895D89AE89BF89988CF02FF81B91E08B
:105420000F1708F090E08F2D821B21E0F81608F08E
:1054300020E0E82FE91B91E08E1708F090E0292B7F
:105440008E2D831B31E0E81608F030E0782F721BB8
:1054500091E0871708F090E0392B8B2D841B21E019
:10546000B81608F020E0682F631B91E0861708F05B
:1054700090E0292B8D2D851B31E0D81608F030E007
:10548000582F521B91E0851708F090E0392B8C2D96
:105490008A1B21E0C81608F020E0482F431B91E04A
:1054A000841708F090E0292B8A2D8B1B91E0A81619
:1054B00008F090E0382F321B21E0831708F020E03D
:1054C000922B1919191BF98BEA8B7B8B6C8B5D8BDB
:1054D0004E8B3F8B188F6D887E888F88988CA9881B
:1054E000BA88CB88DC889501A60160E070E080E096
:1054F00090E002E00E94FC35122FF32EE42ED52E10
:10550000C62EA72E582E392E0E94FC35B22EB10E73
:1055100021E0B11608F020E03F0DE1E03F1508F072
:10552000E0E0422E430E21E0431608F020E0E22B9B
:105530004E0D31E04E1508F030E0EE2EE40E21E085
:10554000E41608F020E0322B5D0D41E05D1508F017
:1055500040E0D32ED50E21E0D51608F020E0422BF6
:105560006C0D31E06C1508F030E0C42EC60E21E061
:10557000C61608F020E0322B7A0D41E07A1508F0CB
:1055800040E0A32EA70E21E0A71608F020E0422B52
:10559000850D21E0851508F020E0542E580E31E0ED
:1055A000581608F030E0232BF32CF90EF20E2B2DB9
:1055B000342D4E2D5D2D6C2D7A2D852D9F2D04E0E3
:1055C0000E94FC35A32FB42F052F162F372E282E1F
:1055D000E22FEB196A96EFAF6A97F1E02E1708F009
:1055E000F0E03A2F3419E1E0A31708F0E0E0B32E21
:1055F000BF1A21E03B1508F020E0E22B4B2F4E199B
:1056000031E0B41708F030E0A42FAE1B21E04A17B8
:1056100008F020E0322B502F5D1941E0051708F00B
:1056200040E0F52FF31B21E05F1708F020E0422B4C
:10563000612F6C1931E0161708F030E0E62FE41BFB
:1056400021E06E1708F020E0322B732D7A1941E02B
:10565000371608F040E0572F531B21E0751708F06C
:1056600020E0422B822D851921E0281608F020E049
:10567000382F341B432F31E0841708F030E0232B00
:105680009F19921B6A968FAD6A97898FBA8EAB8FDE
:10569000FC8FED8F5E8F4F8F98A3ED8CFE8C0F8D5E
:1056A00018A180911D0190911E01892B09F560912F
:1056B00085047091860461157105D1F08091B4055F
:1056C0009091B505892BA1F4A401930197FE07C021
:1056D00022273327A9012619370948095909CB017F
:1056E000A0E0B0E082179307A407B5070CF496C0BA
:1056F00097011092B5051092B405F8948091C305F6
:105700009091C405A091C505B091C605860D971D61
:10571000A81DB91D8093C3059093C405A093C5052A
:10572000B093C6058091C1059091C2058E0D9F1D55
:105730009093C2058093C1058091C1059091C205E7
:1057400097FF2AC08091C3059091C405A091C5051B
:10575000B091C605181619061A061B06ECF48091BE
:10576000C3059091C405A091C505B091C6050197E8
:10577000A109B1098093C3059093C405A093C50501
:10578000B093C6058091C1059091C20588519C4F88
:105790009093C2058093C1058091C3059091C40583
:1057A000A091C505B091C6058093770490937804C5
:1057B000A0937904B0937A048091C1059091C205B9
:1057C00090937E0480937D04789497FE0AC012160D
:1057D00013063CF40894611C711C811C911C285E0A
:1057E0003340D401C30180509048AF4FBF4F805029
:1057F0009040A140B04038F08FEF9FE79093640451
:105800008093630404C070926404609263043093D4
:1058100066042093650482E08093A80580E0C75A5F
:10582000DF4FE2E10C940D3EDB01982F92959F70C3
:1058300023EB30E0F901E90FF11DE491EC938F7057
:10584000280F311DF901849111968C9311971296AE
:105850001C921297CB010895282FDB0164E60E9469
:10586000943D392F822F0E94943D805DFD018193EC
:10587000832F6AE00E94943D805D11968C9311976E
:10588000832F0E94943D905D91831282CD010895F3
:10589000A0E0B0E0EEE4FCE20C94FC3D482FF92ED1
:1058A000E62ED72E862F972F9C01E901E0E1F7E243
:1058B00000E010E0842F9F2DBF010E94A03D262F05
:1058C000842F9F2DBF010E94A03D482FF92E205DFF
:1058D0002993CF016AE070E00E94A03DFB010F5FB9
:1058E0001F4F0430110531F7405D488319828E2D1A
:1058F0009D2DCDB7DEB7E7E00C94183E1F93CF93F4
:10590000DF93EC0120E030E040E050E01881812F8F
:1059100080538A30C8F4CA01B9012AE030E040E07F
:1059200050E00E94753D9B01AC01812F992787FDB6
:105930009095C097AA2797FDA095BA2F280F391FD9
:105940004A1F5B1F2196E2CF203080E0380781E0BC
:10595000480780E0580720F02FEF3FEF40E050E08D
:10596000C901DF91CF911F910895EF92FF920F939C
:105970001F938091590190915A01A0915B01B091C0
:105980005C017C018D017BE0EE0CFF1C001F111FF0
:105990007A95D1F7E826F9260A271B2780915D0121
:1059A00090915E01A0915F01B091600180935901D7
:1059B00090935A01A0935B01B0935C0180916101C7
:1059C00090916201A0916301B091640180935D01A7
:1059D00090935E01A0935F01B09360018091650197
:1059E00090916601A0916701B09168018093610177
:1059F00090936201A0936301B09364019C01AD0197
:105A000063E156954795379527956A95D1F72827ED
:105A100039274A275B272E253F2540275127EF2C82
:105A2000F02E012F11272E253F25402751272093A7
:105A30006501309366014093670150936801B90195
:105A4000CA011F910F91FF90EF900895282F892F81
:105A5000922F0895362F272F692F782FC901089587
:105A6000A0E2B0E0E6E3FDE20C94F73D9C015B01AF
:105A70008E010F5F1F4FC801B9010E94A03ECC24C8
:105A8000DD247601980140E1842E912C8C0E9D1E20
:105A9000F80180818E3291F41082C9010E947E2C1F
:105AA000A0E0B0E08C299D29AE29BF29CC24D82EB6
:105AB000E92EFA2E98012F5F3F4F2BC08823E9F47F
:105AC000CE0101960817190731F4F50110821182F1
:105AD0001282138210C0F8011082C9010E947E2C2C
:105AE000A0E0B0E08C299D29AE29BF29F501808373
:105AF0009183A283B38381E013C0992787FD90959A
:105B0000C0970A9730F0F501108211821282138239
:105B100006C00815190519F00F5F1F4FB9CF80E0B7
:105B2000A096ECE00C94133ECF92DF92EF92FF929E
:105B30000F931F936B01E82E8A01892FBA010E94EF
:105B40002C2C5EE2F52EF801F382B8016C5F7F4FDA
:105B50008E2D0E942C2CF801F782B801685F7F4FD0
:105B60008D2D0E942C2CF801F386B801645F7F4FC5
:105B70008C2D0E942C2CC8011F910F91FF90EF904B
:105B8000DF90CF900895CF92DF92EF92FF920F9324
:105B90001F936B010E94840F7B018C01C6010E9440
:105BA000840F9B01AC012E193F09400B510BB90129
:105BB000CA011F910F91FF90EF90DF90CF90089551
:105BC000A4E0B0E0E6EEFDE20C94FF3D162F072FB7
:105BD0000E94840F20915501309156014091570148
:105BE00050915801260F371F481F591F29833A83A8
:105BF0004B835C83CE0101960E94DC0FAC010097C1
:105C000011F480E00BC0812F902F9C01D901FA0183
:105C100082E101900D928150E1F781E02496E4E069
:105C20000C941B3E1F920F920FB60F9211242F93CC
:105C30008F939F93AF93BF9380916A0290916B0271
:105C4000019690936B0280936A028091C1059091B6
:105C5000C20501969093C2058093C1058091C1054C
:105C60009091C2058C529140ECF01092C2051092B6
:105C7000C1058091C3059091C405A091C505B0915F
:105C8000C6050196A11DB11D8093C3059093C4055F
:105C9000A093C505B093C60581E090E09093C80538
:105CA0008093C705BF91AF919F918F912F910F90D6
:105CB0000FBE0F901F901895A8E2B0E0E2E6FEE25A
:105CC0000C94F13D082F112707FD1095000F111FAF
:105CD000F801E251FD4F85919491F801E555FF4F90
:105CE0004591549125E0A22EB12CAC0EBD1EB501FC
:105CF0000E94CC0EF801E651FD4FE590F490F801BA
:105D0000EA52FD4FC590D4908FE993E00E94F60BC4
:105D10009EA38DA3C7010E94F60B8C0181E893E03E
:105D20000E94F60B98A78FA3C6010E94F60B1C01D8
:105D300088E793E00E94F60B2C0181E27E01089433
:105D4000E11CF11CB7010E942C2CF70101900020EE
:105D5000E9F73197EE19FF09BF010E9483093C0161
:105D60008AE693E00E94F60B4C018FE1B7010E9496
:105D70002C2CF70101900020E9F73197EE19FF096B
:105D8000BF010E9483096C0180E693E00E94F60B3C
:105D90007C01F50101900020E9F73197EA19FB0930
:105DA000C501BF010E9483092DA13EA1020F131F4F
:105DB0002FA138A5020F131F020D131D040D151D71
:105DC000060D171D080D191D0C0D1D1D0E0D1F1D97
:105DD000080F191FC801A896E2E10C940D3EA0E03F
:105DE000B0E0E5EFFEE20C94F53D3C0186E390E087
:105DF0000E941E0A85E391E00E94F60B4C0184E0AC
:105E000093E00E94F60BEC0189E493E00E94F60B0C
:105E10005C01E0E0F3E0859194910E94F60B6C0147
:105E20008BE393E00E94F60B7C0180E00E945C2EE5
:105E30008C0181E00E945C2EC80DD91DCA0DDB1DAE
:105E4000CC0DDD1DCE0DDF1DC00FD11FC80FD91F1A
:105E500081E06816710419F483E692E002C08BE9D0
:105E600092E00E94F60BC80FD91F8FE193E00E94C9
:105E7000F60B6091150370911603C80FD91F88E1C6
:105E8000AE010E947614CDB7DEB7EEE00C94113E61
:105E9000A4E2B0E0EEE4FFE20C94F43D9C01880F34
:105EA000991FBC01F3E0660F771FFA95E1F7680FC1
:105EB000791F61517D4F7093160360931503F901AB
:105EC000E55EFB4FE081E13009F092C0232B19F031
:105ED00007E913E002C007E113E0C80168E173E0DD
:105EE0000E946B3EFC011082E0E0F3E0659174914A
:105EF000C80146E050E00E945D3E892B61F0E2E07F
:105F0000F3E065917491C80146E050E00E945D3E67
:105F1000892B51F468C0E7E06E2E712C600E711E63
:105F2000F8018781882319F480E090E059C081E26C
:105F300094E09A83898381E494E09C838B8373E06B
:105F4000C72ED12CCC0EDD1EEE24FF2465E0862E5C
:105F5000912C8C0E9D1E50E2552E42E0A42EB12CA9
:105F6000AE0CBF1CF501EA52FD4F65917491C3015F
:105F70000E946B3E8C01009779F1F401852D1192FE
:105F80008A95E9F7B8016D5F7F4FC4010E94A03E7A
:105F9000F60180819181B4010E94A03EF501E25199
:105FA000FD4F6591749101C0A895F999FDCFC40189
:105FB00040E250E00E94E83E01501040F80110829B
:105FC0008EEF9FEFE80EF91EC80ED91E9CEFE91662
:105FD0009FEFF90609F0C1CF0E94C40381E090E071
:105FE0000E94EF2E1BC0609115037091160311C023
:105FF000E23079F486E390E00E941E0A84EC90E09F
:106000000E94F60BAC01609115037091160388E1B4
:1060100003C081E140E050E00E947614A496EFE0D6
:106020000C94103EA4E0B0E0E8E1F0E30C94F93DFC
:106030005C016B01CB0160E074E00E944D3EF50114
:1060400081818E010F5F1F4FB8010E942C2C82E0CE
:10605000E82EF12CEC0EFD1EC601B70142E050E027
:106060000E94B53EF5018281B8010E942C2CC60128
:106070000396B70142E050E00E94B53EF5018381EE
:10608000B8010E942C2CC6010696B70142E050E0F0
:106090000E94B53E2496EAE00C94153EAF92BF9262
:1060A000DF92EF92FF920F931F93CF93DF93D82E3F
:1060B0007B01FB01108189E06D2D0E94DF0DA89509
:1060C0004A9BFDCF012F81E00E94920D19E0C0E0B4
:1060D000D0E091E0A92EB12C01C01F5F812F6D2D62
:1060E0000E94A60D802F992787FD90950C2E02C047
:1060F000959587950A94E2F780FD02C080E204C07E
:10610000FE01E852FC4F84910E94760D0E948A0D98
:106110000E94A10E813149F4C5010C2E02C0880FE6
:10612000991F0A94E2F70827D9CF823141F42196CA
:10613000C730D10594F219E0C0E0D0E0CFCF833171
:1061400029F4F7010083C1E0D0E004C0873131F6C3
:10615000C0E0D0E080E00E94920DCE01DF91CF91AF
:106160001F910F91FF90EF90DF90BF90AF90089537
:10617000A0E0B0E0EEEBF0E30C94F83D982E6B015C
:1061800088E0692DA6010E94DF0DF601108690813E
:10619000892F80538A3040F0892F8154863010F047
:1061A00080E002C0892F8753A8954A9BFDCFC82F56
:1061B000DD27C7FDD09581E00E94920D78E0B72ED3
:1061C000AA2400E010E08B2D692D0E94A60D60ED41
:1061D000E62E63E0F62EE00EF11EF701849190E0CA
:1061E0008C179D071CF050E3A52EAC0E8A2D0E9443
:1061F000760D0E948A0D0E94A10E8131A1F4219694
:10620000F701849190E08C179D072CF440E3A42EB5
:10621000C0E0D0E003C030E3A32EAC0EF601E00FE7
:10622000F11FA082D0CF823169F50F5F1F4FB39469
:10623000F601E00FF11F8081992787FD90950E945C
:10624000283E892B19F40F5F1F4FB39408301105B6
:1062500024F028E0B22E00E010E0F601E00FF11F7C
:10626000E0818E2F80538A3040F08E2F815486300B
:1062700010F080E002C08E2F8753C82FDD27C7FDA6
:10628000D095A1CF833119F4C1E0D0E005C08731AA
:1062900009F099CFC0E0D0E080E00E94920DCE01DD
:1062A000CDB7DEB7EBE00C94143EA0E0B0E0EBE538
:1062B000F1E30C94FC3DEC018B01FB01D0800696D0
:1062C0000E947E2CE82EFBE3F817B8F01D82CE0169
:1062D00003960E947E2CF82E8BE38F1570F01A82A5
:1062E000CE010E947E2C883140F4F801D082818357
:1062F000F282E38221E030E002C020E030E0C90118
:10630000CDB7DEB7E7E00C94183EA0E3B0E0EBE8D1
:10631000F1E30C94FD3D8091B6058093DC058091FE
:10632000B9059091BA05A091BB05B091BC058093C9
:10633000DD059093DE05A093DF05B093E005809125
:10634000BD059091BE05A091BF05B091C005809399
:10635000E1059093E205A093E305B093E4050E9464
:106360009E0D80E060E040EE53E00E94CF0D8091F2
:10637000DC05E82FF0E0EE0FFF1FE653FC4F4591E0
:10638000549181E061E00E94CF0D0E94A10E813105
:10639000B9F48091DC058F5F8093DC05833010F0C9
:1063A0001092DC0581E00E94C90D8091DC05E82F88
:1063B000F0E0EE0FFF1FE653FC4F45915491E1CF03
:1063C000833119F0873109F710C11092B805109286
:1063D000B7058091DC05882309F4B2C08E010F5EF9
:1063E0001F4F8DED95E0B8010E941230E1E2EE2ED4
:1063F000F12CEC0EFD1E81EE95E0B7010E941230EB
:106400000E949E0D81E060E049EF53E00E94CF0DB5
:1064100088E060E0A8010E94DF0D80E061E041EFCC
:1064200053E00E94CF0D88E061E0A7010E94DF0DDC
:1064300080E0B8010E94B830892B09F4D6C0C801A9
:106440006DED75E00E945531892B09F4CEC081E0D5
:10645000B7010E94B830892B09F4C7C0C70161EEAB
:1064600075E00E945531892B09F4BFC0B8C09091E6
:10647000DD0548ED53E09A018E010F5F1F4FA0E24A
:10648000BE01695F7F4F90FF05C0F9018491F8015B
:10649000808302C0F801A0832F5F3F4F06171707C4
:1064A00021F095950F5F1F4FEECF18862091E105E3
:1064B000DE01199630E2CD01FA2EE92EBE01615FB0
:1064C0007F4F20FF04C0FA0184918C9301C03C935C
:1064D0004F5F5F4FA617B70719F025951196F1CFBB
:1064E000188A0E949E0D80E060E043E154E00E9423
:1064F000CF0D89E060E08E010F5F1F4FA8010E9461
:10650000DF0D80E061E049E054E00E94CF0D89E0BA
:1065100061E04F2D5E2D0E94DF0D80E06DED75E096
:10652000A8010E944E30892B09F45FC081E061EE22
:1065300075E04F2D5E2D0E944E30892B09F455C019
:106540008091DC058093B6058091DD059091DE0594
:10655000A091DF05B091E0058093B9059093BA054D
:10656000A093BB05B093BC058091E1059091E20535
:10657000A091E305B091E4058093BD059093BE051D
:10658000A093BF05B093C00501C0A895F999FDCFB0
:1065900085E390E06091B6050E94F83E01C0A895A1
:1065A000F999FDCF4091B9055091BA056091BB05AD
:1065B0007091BC0586E390E00E940A3F01C0A89557
:1065C000F999FDCF4091BD055091BE056091BF0581
:1065D0007091C0058AE390E00E940A3F06C0809156
:1065E000DC05813009F043CFABCFE096E6E00C94B8
:1065F000193E1F93482F562F172F862F972F9C0138
:10660000D90124E630E0842F622F0E94943DE82FC8
:10661000842F0E94943D492FF0E0E05DFA4FE49111
:10662000ED93822F6AE00E94943D282F3F5F333024
:1066300051F7852F912F1F9108951F935C9810E0BB
:106640008FEF0E944E081F5F1031D1F75C9A1F91A7
:106650000895A8E0B0E0EFE2F3E30C94F63D5C01AE
:10666000E0910601F0E0E55CFA4F749080E18CBDAA
:1066700083E58CBD5C984B9907C000E08FEF0E94CA
:106680004E080F5F0830D1F7D50116968C918E0118
:106690000F5F1F4FB8010E94F9328B810E944E0894
:1066A0008A810E944E08F50180858F5FB8010E94A3
:1066B000F9328B818F770E944E088A810E944E08A2
:1066C000D5011A96ED90FC901B97ECE6F7E0EE0EE4
:1066D000FF1E90E1C92E97E2D92E86E0882E912CDC
:1066E0008C0E9D1EC701B6010E94A03DE62FC7017A
:1066F000B6010E94A03D7C01F0E0E05DFA4FE4911C
:10670000D801ED938D01C6016AE070E00E94A03DC2
:106710006B010815190531F78D818F770E944E089E
:106720008C810E944E088B810E944E088A810E94B3
:106730004E084B9B38C08091B605882311F40EEFAC
:1067400005C0813011F007EF01C00FEB872D0E94CB
:106750004E08802F0E944E08F50180818E010F5F48
:106760001F4FB8010E94F9328B810E944E088A8126
:106770000E944E08D50112968C91B8010E94F93200
:106780008B818F770E944E088A810E944E08F50106
:106790008481B8010E94F9328B818F770E944E0864
:1067A0008A810E944E085C9A80E18CBD8CBD80E598
:1067B0008CBD2896EDE00C94123E682F88E048E4EA
:1067C00055E00E94CF0D0895E82FF0E0EE0FFF1F77
:1067D000E952FB4F4591549180E061E00E94CF0D5A
:1067E0000895E82FF0E0EE0FFF1FE057FB4F4591B3
:1067F000549180E060E00E94CF0D0895A4E0B0E0E5
:10680000E4E0F4E30C94F93DB82EA62E6A01FA01F7
:1068100080817E010894E11CF11CB7010E942C2CA0
:106820008E010E5F1F4F8B2D6A2DA8010E94DF0D78
:106830008AE30E94760DF6018181B7010E942C2C1B
:10684000C8010E947D0D8AE30E94760DF6018281C7
:10685000B7010E942C2CC8010E947D0D2496EAE00D
:106860000C94153EA3E0B0E0E8E3F4E30C94FC3DA7
:10687000D82E7A018B0140348EE7580785E06807EF
:1068800080E0780738F088E06D2D4FE355E00E94F6
:10689000CF0D2EC0CB01BA0120E13EE040E050E038
:1068A0000E94D63D2983C801B70120E13EE040E0C7
:1068B00050E00E94D63D162F072FF82EE92E2CE32C
:1068C00030E040E050E00E94D63D2A83612F702FD7
:1068D0008F2D9E2D2CE330E040E050E00E94D63D0D
:1068E0006B8388E06D2DAE014F5F5F4F0E94FE33DA
:1068F0002396E7E00C94183E8091BE04813049F461
:106900004091B7045091B8046091B9047091BA04F1
:106910001BC08731E1F48091B3049091B404A0913D
:10692000B504B091B6048F5F9F4FAF4FBF4F19F4BE
:10693000EDE0F5E015C04091AB045091AC046091DE
:10694000AD047091AE0481E00E9432340895883124
:1069500019F4EBE0F5E004C0893139F4E9E0F5E041
:106960004591549188E061E004C088E061E048E42A
:1069700055E00E94CF0D0895AFE0B0E0E2ECF4E303
:106980000C94F53D60901F017090210180902301CF
:10699000A0902B01B0902C010091270110912801AB
:1069A0000F5F1F4F909025018091290190912A013E
:1069B00078E0C72ED12CCC0EDD1E8459984FB6013D
:1069C0000E94482C69E0E62EF12CEC0EFD1E80E0C2
:1069D00060E0A7010E94DF0D8FE20E94760D802FFC
:1069E000B6010E942C2CC7010E947D0D8FE20E94EF
:1069F000760D892DB6010E942C2CC7010E947D0DB9
:106A000080E20E94760D8E010C5F1F4FAA0CBB1C0A
:106A1000AA0CBB1C8DE194E0A80EB91EC801B501FB
:106A20000E944D3EC8010E947D0D80E20E94760DBD
:106A3000E0910601F0E0E75CFB4FE4918E2F0E94AD
:106A4000760D89827A826B8280E061E0AE014F5FD1
:106A50005F4F0E94FE338091B605E82FF0E0EE0F05
:106A6000FF1FE65DFA4F4591549189E061E00E9475
:106A7000CF0D80E20E94760D5F9B02C08EE401C0C4
:106A800086E40E94760D80E20E94760D80910901D5
:106A900090910A01019711F480E501C080E20E9403
:106AA000760D2F96EEE00C94113EA0E1B0E0EBE500
:106AB000F5E30C94FB3D0091A7050E949E0D002379
:106AC00019F40E94BC3494C0013019F580E060E0F4
:106AD00041E40E94EA0D6091DA027091DB0280913C
:106AE000DC029091DD028E010F5F1F4FA8010E9412
:106AF000942D0E947D0D80E061E04DE40E94EA0D3E
:106B00006091DE027091DF028091E0029091E102DB
:106B100024C0023041F580E060E047E40E94EA0DC5
:106B20006091E2027091E3028091E4029091E502AB
:106B30008E010F5F1F4FA8010E94942D0E947D0DB2
:106B400080E061E044E40E94EA0D6091A305709149
:106B5000A4058091A5059091A605A8010E94942DF9
:106B60000E947D0D45C0033009F580E060E043E9F7
:106B700055E00E94DF0D83E00E94E433E0E0EE2E5A
:106B8000E1E0FE2E04E06E010894C11CD11CF70167
:106B900081917F01B6010E94142CAC01802F61E02D
:106BA0000E94DF0D0E5F003191F722C0043001F525
:106BB00085E00E94F1338091090190910A01892BAF
:106BC00021F08091B005882339F088E060E048E446
:106BD00055E00E94CF0D07C00E941005AB01BC011B
:106BE00080E00E94323484E00E94E4330E947C34CE
:106BF0006096E8E00C94173EEF92FF920F93DF93BC
:106C0000CF93CDB7DEB760970FB6F894DEBF0FBE57
:106C1000CDBFA82F002309F461C07E010894E11CB8
:106C2000F11C88E0F70111928A95E9F729833A83EC
:106C30004B835C836D837E83AF83988780E2801B68
:106C4000E82FFF27E7FDF09549815A816B817C8110
:106C5000181684F019861A861B861C8688279927A1
:106C60008E1B9F0B04C0440F551F661F771F8A950C
:106C7000D2F728C0202F332727FD3095DB01CA012A
:106C8000022E04C0880F991FAA1FBB1F0A94D2F7B7
:106C900089879A87AB87BC8704C076956795579597
:106CA0004795EA95D2F78D819E81AF81B88504C062
:106CB000880F991FAA1FBB1F2A95D2F7482B592B63
:106CC0006A2B7B2B4D875E876F87788B29853A856A
:106CD0004B855C856D857E85AF8598898A2F60960A
:106CE0000FB6F894DEBF0FBECDBFCF91DF910F91ED
:106CF000FF90EF900895EF92FF920F93DF93CF9361
:106D0000CDB7DEB760970FB6F894DEBF0FBECDBF2C
:106D1000A82F002309F467C07E010894E11CF11C30
:106D200088E0F70111928A95E9F729833A834B832A
:106D30005C836D837E83AF83988780E2801B4D8167
:106D40005E816F817885E82FFF27E7FDF0951816A3
:106D5000B4F0DB01CA01BB0F880B982FDC018D87D3
:106D60009E87AF87B88B882799278E1B9F0B04C0FF
:106D700075956795579547958A95D2F728C0202F26
:106D8000332727FD3095DB01CA01022E04C0B595DB
:106D9000A795979587950A94D2F78D879E87AF8799
:106DA000B88B04C0440F551F661F771FEA95D2F7B2
:106DB00089819A81AB81BC8104C0B695A7959795CE
:106DC00087952A95D2F7482B592B6A2B7B2B49871D
:106DD0005A876B877C8729853A854B855C856D85CD
:106DE0007E85AF8598898A2F60960FB6F894DEBFAE
:106DF0000FBECDBFCF91DF910F91FF90EF9008951F
:106E0000AEE5B0E0E6E0F7E30C94F13DA8E04E011A
:106E10000894811C911CF4016A2E11926A94E9F77E
:106E200029833A834B835C836D837E838F8398872A
:106E3000CE010996FC011192AA95E9F7A986BA86B6
:106E4000CB86DC86ED86FE860F87188B29843A84F4
:106E50004B845C84ED84FE840F85188969807A8078
:106E60008B809C806DA67EA68FA698AA6D807E8062
:106E70008F809884E114F1040105110509F0B3C372
:106E8000621473048404950408F03DC100E02016E8
:106E900000E0300601E0400600E0500688F41FEFF5
:106EA000211631044104510439F030F048E0E42E59
:106EB000F12C012D112D18C0EE24FF24870114C0E0
:106EC00020E0221620E0320620E0420621E05206B1
:106ED00030F038E1E32EF12C012D112D05C020E119
:106EE000E22EF12C012D112DD201C1010E2C04C076
:106EF000B695A795979587950A94D2F787599E4F8F
:106F0000DC012C9180E290E0A0E0B0E08E199F09B6
:106F1000A00BB10B7C018D01E21AF10801091109E6
:106F2000E114F10401051105A1F10E2C04C0220C9D
:106F3000331C441C551C0A94D2F7A40193010E2C57
:106F400004C0220F331F441F551F0A94D2F780E25A
:106F500090E08E199F096DA47EA48FA498A804C008
:106F600096948794779467948A95D2F7622A732AC5
:106F7000842A952AADA4BEA4CFA4D8A804C0AA0C84
:106F8000BB1CCC1CDD1CEA94D2F7ADA6BEA6CFA6D6
:106F9000D8AA6201EE24FF24CDAADEAAEFAAF8AE99
:106FA000920181012070307009AF1AAF2BAF3CAF56
:106FB000C401B301A70196010E94B43D7B018C017D
:106FC000C401B3012DA93EA94FA958AD0E94B43DFB
:106FD000C901DA013C014D01C401B30129AD3AAD4B
:106FE0004BAD5CAD0E94753D9B01AC018701FF2458
:106FF000EE24ADA4BEA4CFA4D8A8C601AA27BB275F
:1070000057016801A82AB92ACA2ADB2AA216B306A0
:10701000C406D506E0F40894610871088108910857
:10702000A20CB31CC41CD51CA214B304C404D50404
:1070300070F0A216B306C406D50648F40894610899
:10704000710881089108A20CB31CC41CD51CA21A9B
:10705000B30AC40AD50AC601B5012DA93EA94FA994
:1070600058AD0E94B43D7B018C01C601B5012DA92C
:107070003EA94FA958AD0E94B43DC901DA015C0197
:107080006D01C601B50129AD3AAD4BAD5CAD0E94B5
:10709000753D9B01AC018701FF24EE248DA59EA5C3
:1070A000AFA5B8A9A070B070E82AF92A0A2B1B2B4B
:1070B000E216F30604071507C0F40894A108B10806
:1070C000C108D108E20CF31C041D151DE214F304E1
:1070D0000405150550F0E216F3060407150728F419
:1070E0000894A108B108C108D108D30199278827BD
:1070F00086017501E82AF92A0A2B1B2BE9AAFAAAAC
:107100000BAB1CABCFC4211431044104510471F406
:1071100061E070E080E090E020E030E040E050E0AE
:107120000E94B43DC901DA011C012D0100E02016C6
:1071300000E0300601E0400600E0500688F41FEF52
:10714000211631044104510431F028F048E050E0A8
:1071500060E070E017C040E050E060E070E012C016
:1071600020E0221620E0320620E0420621E052060E
:1071700028F048E150E060E070E004C040E150E0F9
:1071800060E070E0D201C101042E04C0B695A7955D
:10719000979587950A94D2F787599E4FDC012C91D9
:1071A000E0E2EE2EF12C012D112DD801C701841B38
:1071B000950BA60BB70B821B9109A109B10900978A
:1071C000A105B10561F464015301A218B308C40814
:1071D000D50831E0632E712C812C912C1EC16F9645
:1071E0008FAF6F97082E04C0220C331C441C551C13
:1071F0000A94D2F7EE2DE81B640153010E2E04C051
:10720000D694C794B794A7940A94D2F7A401930193
:107210006F960FAC6F9704C0220F331F441F551F8A
:107220000A94D2F76DA47EA48FA498A80E2E04C051
:1072300096948794779467940A94D2F784017301A3
:10724000E22AF32A042B152BE9A6FAA60BA71CA702
:107250003201882499249201810120703070219696
:107260000CAF1DAF2EAF3FAF2197C601B501A401F2
:1072700093010E94B43D7B018C01C601B501A401BC
:1072800093010E94B43DC901DA0125968CAF9DAFF0
:10729000AEAFBFAF2597BC01CD0121962CAD3DAD62
:1072A0004EAD5FAD21970E94753D9B01AC018701FA
:1072B000FF24EE24A9A4BAA4CBA4DCA4C601AA2767
:1072C000BB275C016D01AE28BF28C02AD12AA216B7
:1072D000B306C406D50660F525966CAD7DAD8EADC2
:1072E0009FAD2597615070408040904025966CAFCF
:1072F0007DAF8EAF9FAF2597A20CB31CC41CD51CCD
:10730000A214B304C404D50498F0A216B306C406AC
:10731000D50670F4615070408040904025966CAF67
:107320007DAF8EAF9FAF2597A20CB31CC41CD51C9C
:10733000A21AB30AC40AD50AC601B501A401930171
:107340000E94B43D7B018C01C601B501A4019301EB
:107350000E94B43DC901DA013C014D01C401B301F1
:1073600021962CAD3DAD4EAD5FAD21970E94753D90
:107370009B01AC018701FF24EE2489A59AA5ABA54A
:10738000BCA5A070B07057016801A82AB92ACA2A02
:10739000DB2AA216B306C406D506E0F408946108F9
:1073A000710881089108A20CB31CC41CD51CA2143E
:1073B000B304C404D50470F0A216B306C406D506FF
:1073C00048F408946108710881089108A20CB31C64
:1073D000C41CD51C8DA59EA5AFA5B8A96F960FACF2
:1073E0006F9704C0880F991FAA1FBB1F0A94D2F77A
:1073F0008DA79EA7AFA7B8ABA21AB30AC40AD50A35
:107400002596ECACFDAC0EAD1FAD2597D7019927A5
:107410008827682A792A8A2A9B2A820122273327E9
:1074200029960CAF1DAF2EAF3FAF2997A201910156
:10743000407050702D962CAF3DAF4EAF5FAF2D9783
:10744000C601B50129962CAD3DAD4EAD5FAD299776
:107450000E94B43D7B018C01C601B50129962CAD7B
:107460003DAD4EAD5FAD29970E94B43DC901DA0133
:1074700061968CAF9DAFAEAFBFAF6197BC01CD0140
:107480002D962CAD3DAD4EAD5FAD2D970E94753D57
:107490009B01AC018701FF24EE24ADA4BEA4CFA4C0
:1074A000D8A8C601AA27BB2757016801A82AB92A6C
:1074B000CA2ADB2AA216B306C406D50660F5619671
:1074C0006CAD7DAD8EAD9FAD6197615070408040D9
:1074D000904061966CAF7DAF8EAF9FAF6197A20C6D
:1074E000B31CC41CD51CA214B304C404D50498F066
:1074F000A216B306C406D50670F4615070408040F1
:10750000904061966CAF7DAF8EAF9FAF6197A20C3C
:10751000B31CC41CD51CA21AB30AC40AD50AC601DE
:10752000B50129962CAD3DAD4EAD5FAD29970E94BA
:10753000B43D7B018C01C601B50129962CAD3DAD52
:107540004EAD5FAD29970E94B43DC901DA015C01DF
:107550006D01C601B5012D962CAD3DAD4EAD5FADB3
:107560002D970E94753D9B01AC018701FF24EE24FD
:107570008DA59EA5AFA5B8A9A070B070E82AF92A7C
:107580000A2B1B2BE216F30604071507C0F4089418
:10759000A108B108C108D108E20CF31C041D151D97
:1075A000E214F3040405150550F0E216F30604078F
:1075B000150728F40894A108B108C108D1086196FC
:1075C000ECACFDAC0EAD1FAD6197D70199278827B4
:1075D00096018501082B192B2A2B3B2B09AB1AABE3
:1075E0002BAB3CAB62C26E147F048006910608F49C
:1075F00051C220E0E21620E0F20621E0020720E07E
:10760000120788F43FEFE316F1040105110531F08C
:1076100028F048E050E060E070E017C040E050E043
:1076200060E070E012C040E0E41640E0F40640E0A4
:10763000040741E0140728F048E150E060E070E002
:1076400004C040E150E060E070E0D801C701042EC2
:1076500004C0B695A795979587950A94D2F7875950
:107660009E4FDC012C9130E2A32EB12CC12CD12CE9
:10767000D601C501841B950BA60BB70B821B910984
:10768000A109B1090097A105B10589F4E614F70431
:107690000805190508F4F2C16DA47EA48FA498A86A
:1076A000621473048404950408F0E8C1F3C16E9673
:1076B0008FAF6E97082E04C0EE0CFF1C001F111F29
:1076C0000A94D2F76A2D681BD201C101062E04C0AC
:1076D000B695A795979587950A94D2F75C016D01A9
:1076E000AE28BF28C02AD12AADA2BEA2CFA2D8A65A
:1076F000720161016E960FAC6E9704C0CC0CDD1C5C
:10770000EE1CFF1C0A94D2F7C9A2DAA2EBA2FCA2DB
:1077100064015301062E04C0D694C794B794A7946D
:107720000A94D2F7D401C3016E960FAC6E9704C0D1
:10773000880F991FAA1FBB1F0A94D2F7EDA4FEA4BD
:107740000FA518A904C016950795F794E7946A95B4
:10775000D2F737014801682A792A8A2A9B2A6D8E36
:107760007E8E8F8E98A2EDA0FEA00FA118A53801E5
:1077700088249924980187012070307065960CAF99
:107780001DAF2EAF3FAF6597C601B501A4019301B0
:107790000E94B43D7B018C01C601B501A401930197
:1077A0000E94B43DC901DA011C012D01C201B101E1
:1077B00065962CAD3DAD4EAD5FAD65970E94753DB4
:1077C0009B01AC018701FF24EE24AD8CBE8CCF8CD5
:1077D000D8A0C601AA27BB2757016801A82AB92A41
:1077E000CA2ADB2AA216B306C406D50600F50894F9
:1077F0002108310841085108EDA0FEA00FA118A5ED
:10780000AE0CBF1CC01ED11EAE14BF04C006D106F4
:1078100070F0A216B306C406D50648F408942108F1
:10782000310841085108AE0CBF1CC01ED11EA21A5F
:10783000B30AC40AD50AC601B501A40193010E9486
:10784000B43D7B018C01C601B501A40193010E94E6
:10785000B43DC901DA013C014D01C401B301659693
:107860002CAD3DAD4EAD5FAD65970E94753D9B0162
:10787000AC018701FF24EE248D8D9E8DAF8DB8A1C4
:10788000A070B07057016801A82AB92ACA2ADB2A59
:10789000A216B306C406D50600F50894610871085F
:1078A000810891086DA17EA18FA198A5A60EB71E93
:1078B000C81ED91EA616B706C806D90670F0A216AD
:1078C000B306C406D50648F4089461087108810817
:1078D0009108A60EB71EC81ED91ED601C501821B6F
:1078E000930BA40BB50B898F9A8FAB8FBC8FD101F3
:1078F0009927882764015301A82AB92ACA2ADB2AB2
:10790000A9AABAAACBAADCAA860175012FEF3FEF7C
:1079100040E050E0E222F32204231523A60166276B
:1079200077276D964CAF5DAF6EAF7FAF6D97A9A017
:10793000BAA0CBA0DCA06FEF7FEF80E090E0A622A2
:10794000B722C822D92289A19AA1ABA1BCA11D014D
:1079500044245524C801B701A60195010E94753D34
:1079600069966CAF7DAF8EAF9FAF6997C801B701C5
:10797000A20191010E94753D3B014C016D966CADD9
:107980007DAD8EAD9FAD6D97A60195010E94753DB1
:107990007B018C016D966CAD7DAD8EAD9FAD6D970D
:1079A000A20191010E94753D5B016C01A801970144
:1079B000260D371D481D591D69966CAC7DAC8EACEB
:1079C0009FAC6997C401AA27BB27280F391F4A1FFC
:1079D0005B1F2E153F054007510748F4E12CF12CA1
:1079E00061E0062F112DAE0CBF1CC01ED11ECA01B6
:1079F000AA27BB27BC01CD016A0D7B1D8C1D9D1DD7
:107A0000698C7A8C8B8C9C8C661677068806990616
:107A100040F1661577058805990509F043C0D9013D
:107A20009927882769962CAD3DAD4EAD5FAD69971E
:107A300040705070820F931FA41FB51F2DA53EA547
:107A40004FA558A96E960FAC6E9704C0220F331F36
:107A5000441F551F0A94D2F7281739074A075B07B6
:107A600008F509A91AA92BA93CA9015010402040EA
:107A7000304009AB1AAB2BAB3CAB14C06624772467
:107A8000430121E030E040E050E029AB3AAB4BABA2
:107A90005CAB0BC066247724430119AA1AAA1BAA5F
:107AA0001CAA03C0662477244301FE01719688E076
:107AB000DF011D928A95E9F7A9A8BAA8CBA8DCA88E
:107AC000A98ABA8ACB8ADC8A6D8A7E8A8F8A988E46
:107AD00029A93A894B895C89662D7E898F89988D81
:107AE000C25ADF4FE2E10C940D3E629FD001739FBA
:107AF000F001829FE00DF11D649FE00DF11D929F4A
:107B0000F00D839FF00D749FF00D659FF00D992788
:107B1000729FB00DE11DF91F639FB00DE11DF91FAC
:107B2000BD01CF0111240895991B79E004C0991F6C
:107B3000961708F0961B881F7A95C9F780950895C7
:107B4000AA1BBB1B51E107C0AA1FBB1FA617B70783
:107B500010F0A61BB70B881F991F5A95A9F780959F
:107B60009095BC01CD010895A1E21A2EAA1BBB1B62
:107B7000FD010DC0AA1FBB1FEE1FFF1FA217B307F9
:107B8000E407F50720F0A21BB30BE40BF50B661F0F
:107B9000771F881F991F1A9469F7609570958095D3
:107BA00090959B01AC01BD01CF01089597FB092E73
:107BB00005260ED057FD04D0D7DF0AD0001C38F4BC
:107BC00050954095309521953F4F4F4F5F4F089509
:107BD000F6F790958095709561957F4F8F4F9F4FE9
:107BE00008952F923F924F925F926F927F928F9261
:107BF0009F92AF92BF92CF92DF92EF92FF920F933C
:107C00001F93CF93DF93CDB7DEB7CA1BDB0B0FB645
:107C1000F894DEBF0FBECDBF09942A883988488802
:107C20005F846E847D848C849B84AA84B984C88498
:107C3000DF80EE80FD800C811B81AA81B981CE0F8F
:107C4000D11D0FB6F894DEBF0FBECDBFED01089574
:107C5000911106C080538A5010F0865C06C00895CA
:107C600099278827089585FDFBCF80629111F8CF71
:107C700081568A51E0F708959111089581568A51ED
:107C800008F4805285580895FB01DC018D91059020
:107C900080190110D9F3990B0895FB01DC010590BF
:107CA0000D920020E1F70895FC0105900020E9F70E
:107CB000809590958E0F9F1F0895FB01DC01415028
:107CC000504030F08D910590801919F40020B9F7DB
:107CD000881B990B0895FB0155915523A9F0BF010D
:107CE000DC014D9145174111E1F759F4CD010590A3
:107CF000002049F04D9140154111C9F3FB0141119C
:107D0000EFCF81E090E001970895DC0101C06D9311
:107D100041505040E0F70895FC018191861721F011
:107D20008823D9F7992708953197CF010895FB014A
:107D3000DC018D91019080190110D9F3990B089500
:107D4000FB01DC0101900D920020E1F70895FB0199
:107D5000DC014150504030F08D910190801919F4B0
:107D60000020B9F7881B990B0895FB01DC014150F5
:107D7000504048F001900D920020C9F701C01D92BB
:107D800041505040E0F70895DC01CB01FC01F99926
:107D9000FECF06C0F2BDE1BDF89A319600B40D9257
:107DA00041505040B8F70895F999FECF92BD81BD7A
:107DB000F89A992780B50895A6E1B0E044E050E034
:107DC0000C94C63EA8E1B0E042E050E00C94C63E00
:107DD000DC01A40FB51F4150504048F0CB01840F87
:107DE000951F2E910E94F93E41505040D0F70895C2
:107DF000262FF999FECF92BD81BDF89A019700B464
:107E0000021639F01FBA20BD0FB6F894FA9AF99A03
:107E10000FBE08950396272F0E94F93E0E94F83E58
:107E2000252F0E94F93E242F0C94F93EDC01CB0152
:107E300003C02D910E94213F41505040D0F708953A
:107E4000262FF999FECF1FBA92BD81BD20BD0FB676
:107E5000F894FA9AF99A0FBE01960895242F0E9479
:107E6000213F252F0E94213F0C94363F0E94203F46
:0A7E7000272F0C94213FF894FFCF58
:107E7A0002000000000002C010010000000000091A
:107E8A0000010000004600000000000000010000A0
:107E9A000000000900010000004600000000000088
:107EAA000000000000000001000000460000000081
:107EBA000000000000000009000100000046000068
:107ECA000000000000907E000015CD5B07E5559A82
:107EDA0015B53B121F3313490500010202030303C0
:107EEA000304040404040404040505050505050542
:107EFA000505050505050505050606060606060621
:107F0A000606060606060606060606060606060607
:107F1A0006060606060606060607070707070707F0
:107F2A0007070707070707070707070707070707D7
:107F3A0007070707070707070707070707070707C7
:107F4A0007070707070707070707070707070707B7
:107F5A0007070707070707070708080808080808A0
:107F6A000808080808080808080808080808080887
:107F7A000808080808080808080808080808080877
:107F8A000808080808080808080808080808080867
:107F9A000808080808080808080808080808080857
:107FAA000808080808080808080808080808080847
:107FBA000808080808080808080808080808080837
:107FCA000808080808080808080808080808080827
:0A7FDA000808080808080808080055
:00000001FF
